:089BD70033302E322020200063
:0C87EA004109E801C103C100C101C10246
:109663009009007B017A0879EDEBF0A3EAF0A3E916
:10967300F0229000051241A9FF9000061241A9FDB6
:109683009000040241A99000031241A9FF2290090E
:05969300E87401F02263
:10501B0030B60930B7037F2C227F2D2230B7037FA8
:05502B002E227F2F2260
:104504009008E87401F0E4A3F0A3F0A3F0A3F0751D
:10451400FFDE75FFADF5E6F5E71292F1129B04128A
:104524009B4F128AFB12950B12501B9009E9EFF076
:10453400129B7F43F602D2AF200208301405E4FF39
:10454400129A78A2149202127704129700EF605E16
:10455400129077EF24F8601C24F8601D24F0601E8C
:1045640024E0602224C0603A247C703930002A128E
:104574009B1980311297B1800812998F800312978A
:104584005C1298B2801F3000109009E9E0FF7BFFB5
:104594007A9B79D712901F800CE4FF1299AAC20368
:1045A400800312800C129691129700EF70A27B0187
:1045B4007A0879ED129730EF700302473D9008EFC7
:1045C400E0124485462E04464F0545FB1445F0167B
:1045D40045E71746031A46171B46221D46281E00A8
:1045E40000467E9009EAE054FEF0800D9009EAE06E
:1045F4004401F0C2078002D20012969102467E90D6
:1046040008FD129666124190FE9009E9E0FF6E7073
:104614006980059009E9E0FF129AC002467E129B68
:10462400E702467E129C0002467E12966312968929
:104634009009E9E06F7043A3E030E036900900127E
:10464400966C129675FB128C7B80271296631296D9
:10465400899009E9E06F7022A3E030E01590090029
:1046640012966C129675FB1289E09008A8E0FF126E
:1046740048189009E9E0FF129A5F9009EAE020E007
:10468400030245B29008EFE014602B24FA603D1455
:10469400607224F9700302472B240D60030245B2B3
:1046A4001248229008FD12966C1296899008A8F080
:1046B4001299AA0247251248229008FD12966C12FC
:1046C40096899008A8F012481802472512482C90A1
:1046D400090312966C129689129683FD90000512B6
:1046E40041A9FBC003900903E0FBA3E0FAA3E0F9AE
:1046F4009000061241A9900929F0D0031288A11252
:104704009691801D12482C90090312966C1296897A
:10471400129683FD9000051241A9FB1275C01296F2
:1047240091129B980245B27B017A0879ED900906B3
:1047340012966C1283FA0245B230010A9009E9E03C
:10474400FF129A46C20130141AE49008ECF0900863
:10475400ECE0FFC3940F500B1248369008ECE004D1
:10476400F080EB900407E0FF7E00C39455EE9400C4
:104774005007E49008E8F08014C3EF94AAEE940084
:104784009008E850057401F080037402F09008E981
:10479400E0FF9008E8E0FE6F60031296919008E94C
:1047A400EEF09009EAE0C413135403FFBF02209013
:1047B40008D5E0FCA3E0FDD39400EC948040059080
:1047C40008EA8016C3EC9480501A9008EA8010EF2F
:1047D4007012E5289008EA30E7057401F0800A7445
:1047E400FFF08005E49008EAF09008EBE0FF900801
:1047F400EAE0FE6F60031296919008EBEEF09009E8
:10480400E8E06401600302453C124D64E49009E869
:04481400F002453C2D
:10481800129A789009E87401F022129B3E7B017A83
:0E4828000879ED22129B3E7B017A0879ED2281
:10991500E0FEA3E0A60608F6E4F584C2AF43B7016E
:0F99250022E475F001024287EEF0A3EFF0A322D7
:10962C00AB84A2AF9209E4FCFDED9009EC12443C32
:10963C009009EE781D129915438F02438F0118E69D
:10964C00FE08E6F5828E83E4F053B7FEF58FA2098F
:06965C0092AFAF038F8402
:0196620022E5
:02944900AB0571
:10944B00AA84A2AF920AE4FCFDED9009F012443C11
:10945B00EBFF3395E0FEEFF44E601C9009F278625F
:10946B00129915758F0118E6FC08E6F5828C83EBD3
:0F947B00F053B7FEE4F58FA20A92AFAF028F84D1
:01948A0022BF
:108F0F009009B212992DECF0A3EDF0A3EAF0A3EBC8
:108F1F00F09009B6E07002A3E060429009B2E0FE63
:108F2F00A3E0FFA3E0FCA3E0F5828C83E0FD1294A5
:108F3F00499009B7E024FFF09009B6E034FFF090B4
:108F4F0009B5E004F070069009B4E004F09009B39D
:0E8F5F00E004F070BC9009B2E004F080B4228F
:089BDF00E4900000F0A3F02265
:1097D800900000E0FEA3E0FF12962C900000E0FE4F
:1097E800A3E0FF7C007D027B007A04128F0FE490D7
:0697F8000000F0A3F022C6
:0A8B7F00A9059009B8EEF0A3EFF08D
:108B8900EE54FCFE900000E0FCA3E0FD7002EE6CE8
:108B9900604CED4C60031297D89009B8E0FEEE5492
:108BA900FCFE7F00900000F0A3EFF09009BA129943
:108BB9002D7400F0A37402F07E049009BA1299266C
:108BC90085F082F583E493FD9009BC12992685F01E
:108BD90082F583EDF0EF1F70011EEF4E70DC9009F6
:108BE900B8E0FCA3E0FDEC5403FC74022DF582749B
:068BF900003CF583E9F0E9
:018BFF002253
:109548009009A412992DEBF0A3EAF0A3E9F0900991
:10955800A974FFF5F012428745F0601E9009A41225
:109568009926AFF0FE9009A6E0FBA3129926A9F070
:0B957800FA124190FD128B7F80D4227C
:10912700EFF0A3ECF0A3EDF0A3EBF0A3EAF0A3E9D3
:10913700F0227403F0A374E8F0A3E584F0E4F58467
:1091470022D2C4D2C5D2C2C2C3E4900A34F0FF22ED
:10915700E0FBA3E475F001124287A9F0FA22E025AB
:10916700E044A0F5C27F032274FFF5F01242714577
:02917700F022E4
:069BEE00C2C253E6FD2295
:067DF30090091A1291270D
:107DF90090092312913920C7FDC2C4D2C2D2C5E469
:107E0900FF900A34F030C3FDAEC1EE24F86023249C
:107E1900F8601F24F8602924F8603024F8603424BD
:107E2900F87003027EB624F87003027EBE2438027D
:107E39007EC6EF700690091A129165C2C5027ECC02
:107E490090091BE0F5C27F05027ECC900A347403C9
:107E5900F08070EFB4050B90091BA3E0F5C27F0613
:107E69008061EF64067034900922E090091D700565
:107E79001291578008E0FBA3E0FAA3E0F9124190C0
:107E8900F5C2900921E024FFF0900920E034FFF0C9
:107E9900E07002A3E0702C7F078028EFB40706D2B8
:107EA900C47F09801E900A347405F08016900A3444
:107EB9007404F0800E900A347406F08006900A3437
:107EC9007401F0EFB40904C2C38025900A34E0B408
:107ED900030B90092312916F6003129148900A34A1
:107EE900E06008C2C5D2C4C2C38005C2C3027E0E07
:097EF90020C7FD900925E0F58485
:017F0200225C
:064EE70090093212912730
:104EED0090093A12913920C7FDD2C2C2C4D2C5E48D
:104EFD00FF900A34F030C3FDAEC1EE1244854F3041
:104F0D00004F33084F33104F58184F63204F6B2805
:104F1D004F86304F8E384F96404FA6504FCE58008B
:104F2D00004F30024FD4C2C5EF7009900932129173
:104F3D0065024FDAEF64016003024FDA900932E047
:104F4D0025E044A1F5C27F04024FDA900933E0F564
:104F5D00C27F05024FDA900A347403F0806FEFB40C
:104F6D00050B900933A3E0F5C27F068060EFB40610
:104F7D0006D2C57F0180568018900A347404F080E3
:104F8D004C900A347406F08044EFB404047F028020
:104F9D003C900A347405F08034900935129157E530
:104FAD00C21241D6900939E024FFF0900938E0345F
:104FBD00FFF0E07002A3E07004C2C280107F028097
:104FCD000CD2C47F098006900A347401F0EFB40945
:104FDD0004C2C38025900A34E0B4030B90093A1241
:104FED00916F6003129148900A34E06008C2C5D2F7
:104FFD00C4C2C38005C2C3024F0220C7FD90093C45
:03500D00E0F58447
:01501000227D
:10783800900967EFF090096A129130900968ECF0AE
:03784800A3EDF0BD
:10784B00751B00543FF51C543F6058C37440951C86
:10785B00FFE4951BFE90096DE0FCA3E0FDC39FECDC
:10786B009E50068C198D1A80048E198F1A12793C32
:10787B0060037F0222900969E0251AF0900968E005
:10788B003519F090096FE0700B90096BE519851AAB
:10789B00F0124271C390096EE0951AF090096DE0F9
:1078AB009519F090096DE0F519A3E0F51AD3E51AD7
:1078BB009400E51994004076E51A9440E51994007C
:1078CB00500F12793C60037F0222E4F519F51A8000
:1078DB00DC900967E0FFA3E0FCA3E0FDA3E0FBA3C2
:1078EB00E0FAA3E0F9900920E4F0A37440F09009CA
:1078FB006FE0900922F0127DF3900A34E060037F71
:10790B00022274C0251AF51A74FF3519F51990095E
:10791B0069E02440F0900968E03400F090096FE0D2
:10792B00708B90096B75F0401242710278B87F0032
:10793B0022900967E0FFA3E0FCA3E0FDA3E0FBA31B
:10794B00E0FAA3E0F9900920E519F0A3E51AF0900D
:0F795B00096FE0900922F0127DF3900A34E022C8
:109AA900900938E4F0A304F0124EE7900A34E0601C
:079AB900037F01227F002260
:1099C500900A33EBF07B017A0A793390096DE4F064
:0A99D500A304F0E4A3F01278382296
:10989000C00790099AE0FFA3E0900938CFF0A3EF4A
:1098A000F0D007124EE7900A34E060037F01227F78
:0298B000002294
:1099DF00C0079009A2E0FFA3E090096DCFF0A3EFBD
:0A99EF00F0E4A3F0D007127838224C
:1087F6004207590000420644000042063F0000C1FD
:0588060006C105C104DC
:1092600090063FE475F001024271D390075AE094F2
:1092700000900759E06480948022E0FEA3E0244639
:10928000F582740622E490063FF0A3F022E0FBA3EF
:10929000E0FAA3E0F98E827583002290063BE00499
:0992A000F02290063AE004F022ED
:0A9BC400C205C206E4900643F02239
:10993400E4900759F0A3F0900644F0A3F0A3F012CA
:0F994400928690063A04F0A3E4F0900642F022D7
:069BF400129BC40299342B
:109A2D00E4F5848FC343C30175C04475CF8EC2C3A3
:099A3D0043E60290064104F02208
:109B3E00E4F58420C7FDC2C2129BF4E4900641F006
:019B4E0022F4
:0B9B9800E4F584D2C290064104F022E4
:0D9B7F00AE07129A2D90063EEFF0029BF407
:10982400E4900A21F0A3F0300502FF222006FDD2C5
:109834000590063CE4F0A37410F0900747EFF0E4C1
:04984400A3F07F010D
:0198480022FD
:1096980030050A90063CE07002A3E070037F0022C8
:1096A80090063DE024FFF090063CE034FFF0900780
:1096B80048E0FE04F074492EF582E43407F583EFA0
:0496C800F07F01220C
:0B9BA300300507C205D206129B70229D
:0E9B7000AF84E4F58420C7FDC2C4D2C58F8443
:019B7E0022C4
:108D6E009009ACEBF0A3EAF0A3E9F0900641E070B5
:108D7E0002FF229009AFE0FE6005D3941040037FFE
:088D8E000022129824EF60445A
:108D9600E49009B1F09009AFE0FF9009B1E0FEC39D
:108DA6009F501A9009AC12928D1241A9FF12969803
:108DB600EF7002FF229009B1E004F080D8E490063B
:108DC60043F0129BA39009B0E070032006FD9006C5
:048DD60043E0FF2255
:038DDA007FFF22F6
:0E8676009009F4EBF0A3EAF0A3E9F0A3EDF015
:10868400E4FF12926A50012253E6FD90063F1292D3
:108694007A3EF583E0FF129260FCE4B5F007ECB497
:1086A400010312928512929B70031292A2E4FE902F
:1086B40009F7E0FDEEC39D5036EEC39F503190069E
:1086C4003FE0FC12927C3CF583E0FD9009F41292A9
:1086D4008DED1241E8129260FCE4B5F007ECB401B0
:1086E4000312928512929B70031292A20E80C0EE26
:1086F400C39F501A129260FCE4B5F007ECB4010376
:1087040012928512929B70031292A20E80E190073E
:108714005AE024FFF0900759E034FFF043E602905A
:0D87240009F7E0FEEFC39E50028002AF0691
:018731002225
:0C9B8C0012926A40047F0180027F0022D8
:03501800027323FD
:10732300C0E0C0F0C083C082C0D075D000C000C030
:0373330006C0078A
:10733600C20BAFC1EF124485736C08736C10737C7B
:1073460018738120738E2873BB3073C63873CE6072
:1073560073C96873CE7073C97873D68073D6907408
:1073660044A000007452900747E0F5C2C2C59007DA
:1073760046E4F0027454900748802890064374FD52
:10738600F0D2C4D2C5027454900748E0FF90074675
:10739600E0C39F5014E0FF04F074492FF582E434F3
:1073A60007F583E0F5C2027454D2C4900643E4F0B4
:1073B600C206027454D2C590064374FEF002745499
:1073C600027449D204027454900639E4F0027454EB
:1073D600900639E07020E5C2F0E0FFC390063BE07E
:1073E6009F7480F890063AE06480985003129934AE
:1073F600900639E004F090063BE024FFF090063A50
:10740600E034FFF090064412927A3EF583E5C2F02E
:10741600900644129263FEE4B5F00BEEB4010790B9
:107426000644E4F0A3F0900639E014F070209007CB
:107436005AE004F07018900759E004F08010300408
:107446000DC204900746E4F0D2C58002D20B300B81
:107456000EC2C6D2C6C2C5C2C4D2C2C20BC206C200
:01746600C362
:10746700D007D006D000D0D0D082D083D0F0D0E0E3
:0174770032E2
:059BFA00A2C7E433FFE7
:019BFF002243
:1099F9007B01E49009C2F0227422F0A3EFF0A322C4
:0A9A09007B01E49009C2F07D042205
:0E937D009009BEEBF0A3EAF0A3E9F0A3EDF037
:10938B00E49009C3F09009BEE0FBA3E0FAA3E0F977
:10939B00A3E09009AFF09009C2E09009B0F0E4FFB0
:1093AB00128D6EEFB4FF0D9009C3E0FE04F0EEC317
:0693BB00940340D17E0086
:0193C1002289
:0B973000900A18EBF0A3EAF0A3E9F0A8
:10973B007E007F007D101244D8900A18E0FBA3E056
:10974B00FAA3E0F97D10128676EF7002FF227F01FB
:01975B0022EB
:10901F00900953129A017413F0124190900956F06F
:10902F009000011241A9900957F09000021241A936
:10903F00900958F09000031241A9900959F090003F
:10904F00041241A990095AF09000051241A9900904
:10905F005BF09000061241A990095CF07A097953F0
:08906F001299F97D0A02937DBC
:109A46009009F8129A017403F0A374FFF07A097969
:099A5600F81299F97D0402937DD8
:109AC0009009FC129A01741CF0A374FFF07A0979D2
:079AD000FC129A0902937DCC
:109A5F00E4900A00F0A3EFF0A3740AF0A3EFF07AFA
:099A6F000A7900129A0902937DA4
:10880B0001450001420002480000014700014600FB
:0C881B000243000041085E0041086400B8
:1098D400900861E0FBA3E0FAA3E0F92204F0A3748A
:1098E40008F0A37468F022FF90085FEAF0A3EFF099
:0198F4002251
:058C0000900A04EFF0F2
:108C050090085FE0FEA3E0FF2401FDE43EFAA9051C
:108C1500900A057401F0A3EAF0A3E9F0900A0512A1
:108C250098D774019008A86B7008E965827003EA0B
:108C350065837006900A051298E01298D4C003C0A7
:108C450002C001900A051298D7D082D083D0E06B7C
:108C55007008E965827003EA65836019900A04E08B
:108C65008F828E83F0900A05A3E0FAA3E01298EBB9
:058C7500900A04E0F08C
:018C7A0022D7
:109077001298D4C003C002C00190085FE0FCA3E0CF
:10908700F9D082D083D0E064017008E9658270036B
:10909700EC65837003FF802F900861E0FBA3E47504
:1090A700F001124287A9F0FA124190FF1298D47486
:1090B700019008A86B7008E965827003EA65837000
:0790C700069008611298E019
:0190CE00227F
:109700001298D4C003C002C00190085FE0FCA3E03F
:10971000F9D082D083D0E064017008E965827003DB
:0F972000EC65837003FF80071298D4124190FF0D
:01972F002217
:109B04007B017A087968900861EBF0A3EAF0A3E995
:059B1400F01298EB22A5
:1077040090085DE5B0F0E05438FF900867E0FE6F44
:107714006017EE6FFC543060069008657410F090AA
:10772400085DE05438900867F0900865E06037140D
:10773400F0703390085DE0FF900866E06FFCC2AF24
:1077440030E409EF20E4057F10128C00EC30E50CE6
:1077540090085DE020E5057F20128C00D2AF9008F0
:107764005DE0900866F0854245E5B020E2047F01C3
:1077740080027F008F42E542602CE5457004F548A5
:10778400F5490549E54970020548D39420E5489434
:1077940003403A900864E070057F40128C00900822
:1077A400647401F08027E5427023E545601FD3E54A
:1077B40049940AE5489400400FE5499420E548942B
:1077C4000350057F04128C00E4900864F08546475A
:1077D400E5B020E3047F0180027F008F46E5466028
:1077E4002BE5477004F543F5440544E54470020570
:1077F40043D39420E54394034039900864E0700532
:107804007F80128C009008647401F022E546702396
:10781400E547601FD3E544940AE5439400400FE52F
:10782400449420E543940350057F08128C00E490AF
:037834000864F0F5
:01783700222E
:108827004108280041082C0043082200020741089C
:108837002900410825005008000000000000000042
:1088470000000000000000000050081000000000B9
:0C88570000000000000000000000000015
:1091C800900A1BE025E025E02410F582E43408220B
:1091D800F58312443C900A1CE0FEA3E0FF22FF7CCA
:1091E800007D0712420AAC06AD07900A23E0FEA3F1
:1091F800E078032225E025E02400F582E434082203
:0E920800F583E0F8A3E0F9A3E0FAA3E0FB226F
:06997200900825E07016CC
:10997800900A35E584F0E4F58490082504F0D2ECEB
:06998800900A35E0F584B1
:01998E0022B6
:10894600AF84E4F584900829E060030289DD04F031
:10895600900828E0FE5403FDEE1313543FFEC2FFB9
:10896600ED14602714603914605524037069C2A1A0
:10897600D2A0D2A3D2A2E59A20E7FB20FFF830F9D5
:10898600F5EE33333354F8F59B804CC2A2D2A0D215
:10899600A3D2A1E59A20E7FB20FFF830F9F5801372
:1089A600C2A3D2A0D2A2D2A1E59A20E7FB20FFF86B
:1089B60030F9F5EE33333354F84404F59B8018C28E
:1089C600A0D2A3D2A2D2A1E59A20E7FB20FFF830DD
:0989D600F9F5EE4430F59B8F84A5
:0189DF002275
:0350150002821004
:10821000C0E0C0F0C083C082C0D075D000C000C034
:0D82200001C002C003C004C005C006C007B5
:10822D00A2AF920C900828E0FF5403FEEF131354F5
:10823D003F9009C5F0EE7003FF80027F019009C6E3
:10824D00EFF09009C4E584F0758400C2FFEEC3948D
:10825D0003505E9009C8E59BF0E59A20E7FB20FFEF
:10826D00F830F9F5759B0030FFFDC2FF9009C9E5A7
:10827D009BF0EE541F33333354F8FF9009C7E0548D
:10828D00074FF09009C5E0145407FF9009C7E0545B
:10829D00F84FF09009C9E0C4F8540FC868FD900973
:1082AD00C8E0C454F048FC9009C7E0FF1270368056
:1082BD00089009C5E0FF1284E5D2A0D2A3D2A2D2C4
:1082CD00A1900828E004F0D3941F4002E4F0900838
:0F82DD0029E4F0C2FFA20C92AF9009C4E0F5842F
:1082EC00D007D006D005D004D003D002D001D000E6
:0B82FC00D0D0D082D083D0F0D0E03290
:03503000028732C2
:10873200C0E0C0F0C083C082C0D075D000C000C00D
:0787420004C005C006C007DA
:10874900900A23E5BFF0A3E5BEF090082CE0146081
:10875900271460442402704F9008201291F5CEC36B
:1087690013CE13D8F91291E6CEC313CE13D8F92D2F
:10877900FFEC3E900820802B9008261291F5CEC37D
:1087890013CE13D8F91291E6CEC313CE13D8F92D0F
:10879900FFEC3E900826800B900A23E0FFA3E090AF
:1087A900082ACFF0A3EFF090082CE004F0E0C3947E
:1087B900034002E4F090082CE02422F582E4340816
:0C87C900F583E0F5BB900825E4F0C2ED5C
:1087D500D007D006D005D004D000D0D0D082D08329
:0587E500D0F0D0E032ED
:0C85B900900A1BEFF0F9A3ECF0A3EDF02A
:1085C500FFAE04E4FCFDE91291FC129208C31243CC
:1085D500D050271291DDE4FCFD900A1BE0FB1291BF
:1085E500FC1291D8EF24F8FFEE34FFFEE434FFFDD2
:1085F500E434FFFCEB1291CC80341291DDE4FCFDF8
:108605001291C8129208D31243D040271291DDE48B
:10861500FCFD900A1BE0FB1291CC1291D8EF2408C7
:10862500FFE43EFEE433FDE433FCEB1291FCF583FD
:1086350012443C1291C8F583E0FCA3E0FDA3E0FEE3
:10864500A3E0FFE47BFF7AFFF9F8C31243D0500A99
:1086550074FF900A1CF0A3F080131291C8F583A350
:10866500A3E0FFA3E0900A1CCFF0A3EFF01291DD89
:0186750022E2
:10811000505050505050505050505050515151515B
:108120005151515151515252525252525252525334
:108130005353535353535354545454545454555504
:1081400055555555565656565656575757575757CD
:10815000585858585859595959595A5A5A5A5B5B8C
:108160005B5B5B5C5C5C5C5D5D5D5E5E5E5E5F5F41
:108170005F5F6060606161616262626363636464E7
:1081800064656565666667676768686969696A6A7C
:108190006B6B6C6C6D6D6E6E6E6F6F7071717272F9
:1081A0007373747475757677777879797A7A7B7C5E
:1081B0007C7D7E7F7F8081818283848585868788A0
:1081C00089898A8B8C8D8E8F9091929394959697B6
:1081D00098999A9B9C9D9E9FA0A2A3A4A5A6A8A99E
:1081E000AAABADAEAFB1B2B4B5B7B8B9BBBCBEC047
:1081F000C1C3C4C6C8C9CBCDCFD0D2D4D6D8DADC9F
:10820000DEE0E2E4E6E8EAECEEF1F3F5F7FAFCFF93
:10886300420970000042097200004209740000428C
:0A8873000976000041097801C10EEA
:108CF600E0C4F854F0C868FEA3E0C4540F48FFEE81
:108D0600540FFEEF25E0FFEE33FE74362FF5827426
:108D1600503EF583E493FE74019322E0FFA3E0CF77
:108D2600900A25F0A3EF2224ABFFEF7F00FE7C0024
:108D36007D5502421C74102BF58274813AF583E44A
:108D4600937F00FE22900407E0FF7E00C39455EE59
:108D5600940022E0FFA3E0A3CFF0A3EFF022900956
:088D6600EAE013131354072285
:0A9BAE00AF84E4F58475D4948F842D
:019BB800228A
:0A9BB900AF8475840175D4948F8485
:019BC300227F
:10958300128D4B5002801AC3EF94AAEE9400EF5051
:109593000D128D2DC374FF9FFBE49EFA800A24569F
:1095A300FF128D30AA06AB07D3EB94FFEA94004079
:0895B300047A007BFF128D3BDE
:0195BB00228D
:1095BC00128D4B50028016C3EF94AAEE9400EF501C
:1095CC0009128D2DAA06AB07800E2456FF128D3082
:1095DC00C374FF9FFBE49EFAD3EB94FFEA94004024
:0795EC0003E4FAFB128D3BC2
:0195F3002255
:1084E500A984E4F584A2AF920DEFB408004003021D
:1084F50085879084FEF82828730285160285430235
:10850500854D02855702856102851E02856B0285B0
:1085150076128D6430E21E8006128D6430E116C23B
:10852500AF900406E025E0FE900405E033900A25AF
:10853500F0A3CE8048E4900A25F0A3F08044C2AFB2
:10854500900407128D218035C2AF900635128D211A
:10855500802BC2AF900633128D218021C2AF9006C9
:1085650031128D218017C2AF129583EE128D2680B0
:108575000CC2AF1295BC900A25EEF0A3EFF0A20D48
:1085850092AF900A25E0F59B30FFFDC2FFE59A20EA
:10859500E7FB20FFF830F9F5900A26E0F59B30FF60
:1085A500FDC2FFD2A0D2A3D2A2D2A1A20D92AFAF9B
:0385B500018F84AF
:0185B80022A0
:035033000271B750
:1071B700C0E0C0F0C083C082C0D075D000C000C09E
:0D71C70001C002C003C004C005C006C0071F
:1071D400900A36E584F0C2CF758403128E493012CA
:1071E40017C392129009EAE0135403FFBF010990F8
:1071F4000974E4F0A3F0806E9009EAE0F9C3135433
:1072040003FF6402703B900974E0FCA3E0FDC3EC4F
:1072140094E04002D20E300E4D900970E0A320E7B6
:1072240045A3E0A330E73FD3ED94FFEC941F400661
:10723400A3E094E04030900974E4F0A3F0C20E801F
:1072440025EF64037020900974E020E7047F018037
:10725400027F00900970E020E7047E0180027E0036
:10726400EE6F24FF9290900974128CF6FDAC0678B0
:1072740005C333CE33CED8F9FDAC068C28F529EC02
:107284006480FC900970128CF6FBAA067805C3335F
:10729400CE33CED8F9FBAA06EA6480FA758400EDF1
:1072A400F5D2ECFF8FD3758401AF03EFF5D2AE02B4
:1072B400EEFF8FD3900970128D59900971E0252D3E
:1072C400F0900970E0352CF0900974128D59A3E008
:1072D40014F07024900975E0252BF0900974E035C2
:1072E4002AF09009EAE0C41313540370047F048065
:1072F400027F01900978EFF0129972128946900A80
:0473040036E0F584F6
:10730800D007D006D005D004D003D002D001D000D9
:0B731800D0D0D082D083D0F0D0E03283
:109787007864E0FEA3E0A60608F6227868E0FEA368
:10979700E0A60608F622E6FE08E6F5828E83229208
:0A97A700AFAF028FB1AF038F842231
:1090CF00AB84AAB1A2AF920F900A0812443C900A47
:1090DF000A12978753B10F900A09E0700543B11038
:1090EF008019900A0AE030E70543B130800D43B193
:1090FF0020900A0AE04480F0129787E4F584C2AF0B
:10910F0043B701758F03786412979DE4F053B7FE50
:07911F00F58FA20F1297A6C5
:019126002226
:108DDD00AB84AAB1A2AF921090097E12443C9009C7
:108DED007DE0F9FF3395E0FEEFF44E604990098088
:108DFD00786612978953B10F90097FE0700543B1E2
:108E0D0010801B900980E030E70543B130800F439F
:108E1D00B120900980E04480F07866129794E4F5D3
:108E2D0084C2AF43B701758F01786612979DE9F043
:0B8E3D0053B7FEE4F58FA2101297A6B9
:018E48002207
:0F8F6D0090093DEBF0A3EAF0A3E9F0A312443C16
:108F7C00E4900946F0A3F0900944E0FEA3E0FFC39F
:108F8C00900947E09F900946E09E502D90094012B1
:108F9C0044071292A990093DE0FBA3E475F001127D
:108FAC004287A9F0FAEF1241D6900947E004F0701D
:098FBC00C6900946E004F080BEF5
:018FC5002289
:1092A900AB84AAB1900A0C12443C900A0E12979210
:1092B90053B10F900A0DE0700543B1108019900A5F
:1092C9000EE030E70543B130800D43B120900A0E1E
:1092D900E04480F0129792786812979DE493FFAE6C
:0792E900028EB1AE038E847A
:0192F000225B
:1092F100900A277427F0A37410F0900A2774FFF5E1
:0F930100F0124287FED3E5F09400EE940050EB9B
:109310007D017F04128EAD129AD7129B2C129BAE48
:10932000129BB9129AEE75F7047FD77E0512984901
:07933000E4F58475D103226E
:108EAD00AE8475840F758C20E4F58475EF0675849A
:108EBD000F758A83F59775840F758904F58475B7D9
:108ECD003075840F4389018D8D758F018F8EFDFC5B
:108EDD000DBD00010CE4B505F7ECB401F3438902B7
:108EED00E58920E4120DEDAA0470010C14D3940051
:108EFD00EA6480948140E9759702E4F58AAF068FA4
:018F0D0084DF
:018F0E002240
:109AD700AF8475840F75E10375E3C043A50175A6CF
:069AE700FF75A4E78F8467
:019AED002256
:109B2C00E4F584759A73759D1843E60175F801C2C6
:029B3C00FF2206
:109AEE00AF84E4F584F5BA75BC9875E88143E70256
:059AFE0043F7028F8414
:019B0300223F
:10984900AD84758402E4F5C875C908C39FFFE49E19
:10985900F5CB8FCA74FFF5CDF5CC43E704D2CAAF77
:03986900058F84E4
:01986C0022D9
:045011000004020194
:1095F400FCA3E0FDEC4EFFEDCF900A2BF0A3EFF0BF
:1096040022E054FEFEA3E0547F4480FF900A2BEE38
:1096140022FEA3E0547FFFEE4401900A2B22900A1D
:089624002BE0FEA3E054F0224C
:104D64003000069009EAE08004A203E4335401C44D
:104D74003333335480FE900A2BE0547F1295F49021
:104D840009EAE0FDC3135403905011935407C4542B
:104D9400F0FE900A2BE0548FFAA3E0FBEA4EFFEBFF
:104DA4001295FCED131313540725E0FE900A2BE033
:104DB40054F11295F49009EAE0FFC413135403F973
:104DC40074017E00A801088005C333CE33CED8F920
:104DD4005407C4F8540FC868FFE4C454F048FE9064
:104DE4000A2BE0FCA3E0548FFDEC4EFEED4FFFEEEA
:104DF4001295FD900407E0FD7C00C39455EC9400EB
:104E04005007129622440C8012C3ED94AAEC94002D
:104E14001296225004440980024403FF900A2BEEA8
:104E2400F0A3EFF0E9640270289008D5E0FCA3E059
:104E3400D39400EC94804008900A2B1296058027A6
:104E4400C3EC9480900A2BE054FE502712961580F0
:104E540016E97019E528900A2B30E70512960580AB
:104E640006E054FE129615F0A3EFF0800C900A2B86
:104E7400E054FEF0A3E0547FF0C287C285E4FD90C5
:104E84000A2BE0FEA3E0A805088005CEC313CE13C9
:074E9400D8F9139286D285C4
:104E9B00E4900A29F0A3F0900A2AE004F07006903F
:104EAB000A29E004F0900A29E07004A3E064017081
:014EBB00E610
:024EBC00C285AD
:104EBE00E4900A29F0A3F0900A2AE004F07006901C
:104ECE000A29E004F0900A29E07004A3E06401705E
:014EDE00E6ED
:074EDF000DEDB4109FD28716
:014EE60022A9
:109A9100000002AB055508000AAB0D55100012ABD2
:089AA100155518001AAB1D5504
:07887D00C1124209D40032D0
:10986D009009CEE4F0A322900A1EE0FBA3E0FAA338
:10987D00E0F9229009CA12443C9009CA22900005D1
:03988D000241A9EC
:107CD600EF75F00C84E5F0FD12986DEDF0EF75F0A0
:107CE6000C8424FFFFE434FFFE9009CEE0FCA3E001
:107CF600FDEC6003027D9EEDB40C004003027D9E08
:107D0600907D0DF8282873027D31027D3A027D426E
:107D1600027D4A027D52027D5A027D62027D6A021E
:107D26007D72027D7A027D87027D9212986D7403C0
:107D3600F0027DA212986D7404F0806012986D7442
:107D460005F0805812986D7406F0805012986D7484
:107D560007F0804812986D7408F0804012986D7490
:107D660009F0803812986D740AF0803012986D749C
:107D76000BF08028E49009CEF0A3F00FBF0000803E
:107D86001B12986D04F00FBF0000801012986D74DE
:107D960002F00FBF00008004E4FEFF22EF7F00C464
:107DA6003354E0FEE4FCFD129880E0F8A3E0F9A36A
:107DB600E0FAA3E0FB9009CFE025E0FF9009CEE0D2
:107DC60033FE74912FF582749A3EF583E493FE7424
:107DD6000193FFE4FCFDEB2FFFEA3EFEED39FDECDF
:0C7DE60038FC129880A3A3E0FEA3E0FF8D
:017DF200226E
:0B83FA00900A1EEBF0A3EAF0A3E9F0EC
:108405001298749000031241A9FD540FFC9009E9DC
:10841500E05403FF74087E00A807088006CEA2E793
:1084250013CE13D8F8FFECFBEF5B24FF9211ED544C
:10843500F02450602124D06052245060030284E46B
:108445002011030284E412987412988AFF127CD6D4
:10845500129BCED212222011030284E412987412C8
:10846500988A641F70799000061241A9FF7E0090DA
:1084750009D4EEF0A3EFF0D39433EE94004060E01E
:1084850024FFF09009D4E034FFF022301151129806
:10849500749000061241A925E09009D2F0A3E4F0FA
:1084A50012988A75F004A4FF9009D2E045F0FEA366
:1084B500E04FFF9009D2EEF0A3EFF02401FFEE3478
:1084C500809009D0F0A3EFF09009D0E0FEA3E0780A
:0F84D50003CEA2E713CE13D8F8F0EE9009D0F043
:0184E4002275
:109B4F009009EAE054FEF054F9F054C7F0543FF096
:019B5F0022E3
:109B19009009EAE020E0044401F0229009EAE054C7
:039B2900FEF02229
:1097B1009009EAE0FFC313FEEF54F9FFEE045403EE
:1097C10025E04FFFF0E0C3135403FEEF54F9FFEE21
:0797D100540325E04FF022D4
:10998F009009EAE0FF131313541FFEEF54C7FFEEC5
:0B999F0004540733333354F84FF02218
:10975C009009EAE0FFC413135403FEEF543FFFEEED
:10976C00045403C4333354C04FF0E0FFC4131354F8
:0B977C0003D394024004EF543FF0229E
:107A92000204FFFFFFFF03050100070906080AFFB2
:107AA200FFFFFF0DFF0B0E0C000100020004000897
:107AB2000010002000400000010202030404050639
:107AC20007070809090A0B0C0C0D0E0E0F101111F5
:107AD200121314141516171718191A1A1B1C1D1E27
:107AE2001E1F202121222324252526272829292A51
:107AF2002B2C2D2D2E2F3031323233343536373771
:107B020038393A3B3C3D3D3E3F4041424343444588
:107B1200464748494A4B4B4C4D4E4F505152535495
:107B22005556565758595A5B5C5D5E5F6061626399
:107B32006465666768696A6B6C6C6D6E6F70717292
:107B42007374757778797A7B7C7D7E7F808182837E
:107B52008485868788898A8B8C8E8F909192939464
:107B6200959697989A9B9C9D9E9FA0A1A3A4A5A63B
:107B7200A7A8A9ABACADAEAFB0B2B3B4B5B6B7B906
:107B8200BABBBCBDBFC0C1C2C4C5C6C7C8CACBCCC4
:107B9200CDCFD0D1D2D4D5D6D8D9DADBDDDEDFE174
:107BA200E2E3E5E6E7E8EAEBECEEEFF0F2F3F5F616
:067BB200F7F9FAFBFDFEED
:10888400C1144204020000420637000041040400FF
:104B3300E4F557E55325E0FFE55233FE74AA2FF55C
:104B430082747A3EF583E493FE740193FFF556E590
:104B530058540FF554E55954F0F55575C30385546E
:104B6300C28555C1759208759100C281C28185962F
:104B73005485955574B82555F582747A3554F58363
:104B8300E493755800F55975C3018558C28559C119
:104B930022E550540FF54CE55154F0F54D75C30320
:104BA300854CC2854DC1759208759100C281C28141
:104BB30085964C85954D74B8254DF582747A354CA0
:104BC300F583E493755000F55175C3018550C28593
:104BD30051C122FBAA06E0FEA3E0FFEF2BFFEE3A52
:104BE300FEE433FDE433FCA312443CE47FFF7EFF89
:104BF300FDFC22759200759140C281C28185945853
:104C0300859359E5594257E558425622EF75F017F7
:104C1300A4241DF582E5F03404F58322C281C28108
:104C2300859450859351E551424FE550424E75505E
:104C33003775510075C301854EC2854FC1855092AA
:104C4300855191C281C281859650859551223480C8
:104C5300AD07FCE0C313FEA3E01375C30E8CC28D36
:104C6300C18E92F59175C27F75C1FF22900A13E040
:104C730075F017A42419F582E5F03404F58322FDB9
:104C8300ECC4F854F0C868FAEDC4540F48FBECC305
:104C930013FEED132BFDEE3AFCE01313543F7E009D
:104CA3002D22E0FEA3E0FF8E928F91C281C281C2CA
:104CB300812275590075C3018556C28557C1855830
:104CC30092855991C281C28185965885955922E072
:104CD300F8A3E0F9A3E0FAA3E0FB228524C285252B
:104CE300C1852C92852D912275F017A42409F58294
:104CF300E5F03404F58322759200759108C281C2F0
:104D030081859652859553E5536407455222900851
:104D1300DFE0C313FEA3E013229009D1E02FF52FA8
:104D23009009D0E03EF52E22900A11E0FEA3E0FFA9
:104D330022E0FCA3E0FDA3E0FEA3E0FF22A4241EE7
:104D4300F582E5F03404F58322E0FEA3E078032244
:104D530085245885255975C30322A3A3E0FFA3E047
:014D6300222D
:10950B00E4900A37F0900A37E0FB124C7312444890
:10951B0000000000EB124C10E4F0FF900A37E01251
:10952B004CEB75F002EF124479E4F0A3F00FEFB4BB
:0C953B0008E9900A37E004F0E0B40FC922
:019547002201
:0B703600900A10EFF0A3ECF0A3EDF0C7
:10704100A2AF9213900A10E0FF907A9293900A13E4
:10705100F0F4703EEFB4120F900A11E0FCA3E0FDD2
:10706100E4FF1285B98017900A10E0B4140DA3E073
:10707100FCA3E0FD7F011285B98003124D2B900A1C
:1070810010E025E0242DF582E43408F583EEF0A329
:10709100EFF0124C6FC083C082124D34C006C0079E
:1070A100900A13E0FF124CEBC083C082124C0FE038
:1070B1005407D082D08375F002124479E0FEA3E038
:1070C100FBAA06D007D006C3EF9BFFEE9AFEED9414
:1070D10000FDEC9400FCD082D08312443C124C6F32
:1070E100C083C082124CD2124D2BE4FCFDEB2FFF6A
:1070F100EA3EFEED39FDEC38FCD082D08312443CEF
:10710100900A13E0FB124C73124D3478031243E1E1
:1071110075F017EB124D40EEF0A3EFF0124D2BA3DB
:10712100E0FD124CEBC083C08275F017ED124C13D9
:10713100E0D082D08375F002124479EEF0A3EFF033
:10714100900A13E0FF124C10E004F0124C0FE054CF
:1071510007F0201460900A13E0FF124C10E0705504
:10716100900403E004F07006900402E004F0900A39
:1071710013E0FE75F017124D40E0FCA3E0FDEE2593
:10718100E024C4F582E43407F583ECF0FCA3EDF0D0
:10719100FDEF25E024A6F582E43407F583ECF0A3A6
:1071A100EDF0C3900403E0943C900402E064809409
:0571B100804002D21431
:0171B60022B6
:108E4900900404E0FF75F00584E5F014603D1460BA
:108E59003F14604114604324047042EF75F00784A5
:108E6900E5F014601214601E1460111460132404D8
:108E7900702B129216802612948B80211294CB802B
:108E89001C12940680171291798012127F03800DAB
:108E9900128A768008127BB88003127478900404D1
:038EA900E004F0F2
:018EAC0022A3
:04933700AD07AC06CC
:10933B009008E1E0FEA3E07806CEC313CE13D8F974
:10934B002401FFEE34FEFED3EF9400EE6480948094
:10935B00400FEF2DFDEE3CFC30E7127C7F7DFF8054
:10936B000CEF2DFDEE3CFC30E703E4FCFDAE04AF4F
:01937B0005EC
:01937C0022CE
:107478009009EAE030E03B9009D4E0FEA3E0FF6425
:10748800324E6022EF24CEFFEE34FFFEEF7802C3C7
:1074980033CE33CED8F9FDAC06124D112DFFEE3C9C
:1074A800FE124D1C8023124D11FF124D1CAF2FFEF2
:1074B80080109008DFE0C313F52EA3E013F52FFF2B
:1074C800AE2E1293378E2E8F2F9008E6E02400F50B
:1074D800359008E5E03480F5349008E3124D4CCE41
:1074E800C313CE13D8F9F5338E32900827E0255F01
:1074F800FF900826E0355E6480F5308F319008559E
:10750800E0FCA3E0900855124C82F537EE3CF536C6
:1075180030E70675367F7537FFC3E537955BF53776
:10752800E536955AF53630E705E4F536F53790092E
:10753800EAE0FF30E0159009D4E07004A3E064327B
:107548006009E4F530F531F536F53775C30E853049
:10755800C28531C18532928533918534C28535C162
:10756800853692853791124C68852E92852F911217
:107578004CAE85CF2685CE27EF131313540730E082
:107588002C75C30E124C688526928527918528C2D2
:107598008529C1900405124D4CCEC313CE13D8F9DA
:1075A8008E92F591124CAE85CF2685CE27E52630F2
:0775B800E705E4F526F527C5
:0175BF0022A9
:108A7600852650852751C3E550648094805005E4CF
:108A8600F550F55175C303124BCF759200759108D9
:108A9600C281C28185964A85954BE54B6407454A56
:108AA6007018F54F754E40124B94759200759140B3
:108AB600124C1F85502C85512D22E4F54FE54B2590
:108AC600E0FFE54A33FE74AA2FF582747A3EF583F9
:108AD600E493FE740193FFF54E124B948E928F91A0
:108AE600124C1FE550A2E713F550E55113F55185D9
:048AF600502CF52DDE
:018AFA002259
:107BB8009009EAE0C413135403146036146078245F
:107BC800026003027CD5124D53124B8D124CFA7091
:107BD80011F557755640124B52124BF67558020262
:107BE8007C13124B338E928F91124BFC7558020204
:107BF8007C2A124D53124B8D124CFA7018F557759A
:107C08005640124B52124BF6755837124CB58558E0
:107C18002A85592B22124B338E928F91124BFC7569
:107C28005837124CB5E558A2E713F558E55913F53E
:107C38005985582AF52B22E52525E0F525E5243335
:107C4800F52430E72063248075C30E124CDE124CF5
:107C5800DE124CDE124C68124CE4124CAE85CF2A70
:107C680085CE2B804575C30EC374FF9525FF747FA1
:107C78009524F5C28FC1124CE4124CAE85CF2A85EB
:107C8800CE2BE52BAE2A7802CEC313CE13D8F9FD3E
:107C9800AC06E52AC313FEE52B132DFFEE3CFEC30D
:107CA800E52D9FF52BE52C9EF52AD3E52B9480E551
:107CB8002A941B4007752A1B752B8022C3E52B9439
:0D7CC8001CE52A94005006752A00752B1C3F
:017CD500228C
:107F03009008D7E0FEA3E07806CEC313CE13D8F9CA
:107F13002401FDEE34FCFC9008D5124D142DFFEC2A
:107F23003EFE900638E02FF539900637E03EF538EF
:107F33009009EAE0C3135403FFBF033074402539AB
:107F4300F53974053538F53890082AE0FEA3E07852
:107F530005CEC313CE13D8F9FFC3E5399FF539E531
:107F6300389EF53830E705E4F538F5399008DCE05C
:107F73002400F53F9008DBE03480F53E9008D912E9
:107F83004D4CCEC313CE13D8F9F53D8E3C9008214A
:107F9300E02561FF900820E035606480F53A8F3B6F
:107FA300900851E0FCA3E0900851124C82F541EE99
:107FB3003CF54030E70675407F7541FFC3E54195C9
:107FC3005DF541E540955CF54030E705E4F540F5A6
:107FD3004175C30E853AC2853BC1853C92853D916F
:107FE300853EC2853FC1854092854191124C68858B
:107FF3003892853991124CAE85CF2485CE25E52460
:0880030030E705E4F524F52542
:01800B002252
:109216009008CBE0C313FFA3E013900A2DCFF0A371
:10922600EFF09008CAE02400FF9008C9E0900833E8
:10923600124C51900A2D124CA5900405E5CFF0A3CF
:10924600E5CEF0E02401F0900405E034FFF0E030D4
:09925600E707E4900405F0A3F021
:01925F0022EC
:109179009008CDE0C313FFA3E013900A2FCFF0A30B
:10918900EFF09008D0E02400FF9008CFE09008317C
:10919900124C51900A2F124CA5900631E5CFF0A33D
:1091A900E5CEF0900631E030E707E4900631F0A310
:0E91B900F0900632E025E0F0900631E033F051
:0191C7002285
:10948B009008DDE0FFA3E09009D6CFF0A3EFF090BA
:10949B00084BE0FEA3E09009D6124BD69009D812E8
:1094AB004CD2D31243D0400974FF900407F0A3F0C1
:0F94BB00229009D8124D5D900407CFF0A3EFF077
:0194CA00227F
:1094CB009008D1E0FFA3E09009DCCFF0A3EFF09080
:1094DB000837E0FEA3E09009DC124BD69009DE12B0
:1094EB004CD2D31243D0400974FF900633F0A3F053
:0F94FB00229009DE124D5D900633CFF0A3EFF003
:01950A00223E
:109406009008D3E0FFA3E09009E2CFF0A3EFF0903D
:109416000835E0FEA3E0FBAA069009E2124BD990BC
:1094260009E4124CD2D31243D0400974FF9006359A
:10943600F0A3F0229009E4124D5D900635CFF0A31B
:02944600EFF045
:019448002201
:099BCE009008DFEEF0A3EFF02295
:109B600000000000000000000000000000000000F5
:0A889400C1074108A8004108E700F1
:10796A0090094FE075F01FA42401F582E5F034F088
:10797A00AF82229009EAE0FF5406FE9008C8E0545C
:10798A00F94EFEF0EF5438FFEE54C74FFFF090095E
:10799A00EAE09008C854C0FEEF543F4EF022A3E03C
:1079AA00FCA3E0FDA3E0FEA3E0FF78040243E17B31
:1079BA00017A0879A9E4F0A322FBE0FEA3E0FFC361
:1079CA00E49FFF74809EFE3395E0FDFCEB2FFFEAF7
:1079DA003EFE22FE7A0879C87B019009A9E4F0A349
:1079EA0022E0F8A3E0F9A3E0FAA3E022900855E028
:1079FA00FCA3E0FDECC4F854F0C868FAEDC4540FD7
:107A0A0048FB22AFF0FEE0FCA3E0F5828C83E4930E
:107A1A00FD2290094BF0A3EFF0E4900951F0A3F096
:107A2A0022EFF0A3EDF0A3EBF0A2AFE433A3F0C290
:107A3A00AF227EF37FA37B007A00795A22EF25E0FA
:107A4A0024C9F582E43408F5832275F01FA42401C1
:107A5A00F974F035F0FA22E475F001024287ED3943
:107A6A00FDEC38FC02443CE93DFDE83CFC02443CA8
:107A7A00900952E004F022900951E004F022FDED51
:087A8A00FFEEF0A3EFF0E4228F
:069C0000E49008E7F022E9
:079BE7009008E77401F02271
:1097FE009008C8E0FF5406FE9009EAE054F94EFEC8
:10980E00F0EF5438FFEE54C74FFFF09008C8E090C9
:06981E0009EA12799F2205
:049C0C0012797D222A
:108FC60012797DE4FFEF600D64036009EF640960C8
:108FD60004EFB40E0B127A477480F0A3E4F0800716
:108FE600127A47E4F0A3F00FEFB40FD9129BDFE437
:108FF600900A38F0900A38E0FFC3941E501875F0B6
:109006001FEF1279711279DD741FF0129548900ADC
:0990160038E004F080DE0297D876
:1096CC00900A317402F0E4A3F0129BDF7EF07F006D
:1096DC007A0A79311279E204F01295487EF37FAB65
:1096EC007B017A0A79321279E404F01295481297C8
:0496FC00D8028FC63B
:1098B20020071E3000119009EAE030E00C9008E722
:1098C200E07006D2018002D2039009E87401F0D25E
:0298D20007226B
:10800C00780A7C097D017BFF7A9B79607E007F106A
:10801C0012416AA2AF9215D2AF3014FDC2AFE490F8
:10802C000909F090090A1279EBFBC000C002C003E9
:10803C001279F6ECC313FEED132BFDEE3AFC90080F
:10804C0055E01313543F7E002DFFEE3CFEE4FCFD87
:10805C00D003D002D0001279D690090A127A689017
:10806C00090E1279EBFBC000C002C0031279F69026
:10807C000851E0C313FEA3E0132BFBEE3AFAEC130A
:10808C0013543F7E002BFFEE3AFEE4FCFDD003D0F0
:10809C0002D0001279D690090E127A689009121249
:1080AC0079EB9008261279C3900912127A71900913
:1080BC00161279EB9008201279C3900916127A7176
:1080CC00900909E004F0E06410600302802F90092D
:1080DC000A1279A98E5A8F5B1279A88E5C8F5D1269
:1080EC0079A88E5E8F5F1279A88E608F61129BDFEC
:1080FC00127A3C1279E47408F01295481297D8A2BF
:03810C001592AF1A
:01810F00224D
:108AFB0090F3ABE493F4600990F000E493640260AC
:018B0B002643
:108B0C00A2AF92161296CCD2AF3014FDC2AF129B0C
:108B1C00DF127A3C1279E47408F01295481297D857
:048B2C00A21692AF4C
:028B300080447F
:108B32007BFF7AF379A3AF01AE027DFF7C00900A3E
:108B42001412443C900A14A3A3E0FEA3E0FFE4FD48
:108B5200FC900A1412443C127A40900A14E0FCA3DE
:108B6200E0FDA3E0FEA3E0FF900944E4F0A3740853
:048B7200F0128F6D01
:098B7600129A13E49008A8F02201
:1098F5009008A8E0FFC3941E5015EF127A547BFF21
:1099050078C87C087D017E007F1F12416AC207224C
:109953009008A8E0C3941E5015129BDF9008A8122C
:0F996300796D1279DD741FF01295481297D82292
:069C0600129953C207226F
:0299AA00AD0707
:1099AC00A2AF9217C2AF129C0C9008A8EDF0129CBB
:0899BC0006129A13A21792AFE4
:0199C4002280
:109A7800A2AF9218C2AF9008A8EFF01298F512970B
:089A8800FE129A13A21892AF1E
:019A900022B3
:0888A100900927EDF0A3EBF0B4
:1088A900A3E004F090092CEFF0A3EBF0900927E086
:1088B900FF90092CE0FED39F506C75F01FEE1279E2
:1088C9007190092EF0A3EFF090092D12796D90099E
:1088D90030F0A3EFF0E490092AF0A3F090093012E8
:1088E9007A6190092E127A0D128B7F90092FE0047C
:1088F900F0700690092EE004F090092BE004F07066
:108909000690092AE004F0C390092BE0941F90090E
:108919002AE0940040C61297D890092CE004F0A3ED
:10892900E004F00288B59008A8E0FF900928E0D398
:0C8939009F5009A3E0C39F4003129A78EE
:01894500220F
:0F75C000900949EDF0900948EFF090094AEBF07F
:1075CF0090094FEFF0A3EBF0900949E0FF90094FBE
:1075DF00E0D39F40030276BAA312796D127A1C9002
:1075EF000951E0FEA3E0FFC3941FEE9400502A90D0
:1075FF00094B127A1074A92FF582E43408F583ED44
:10760F00F090094CE004F0700690094BE004F01282
:10761F007A7A70CB127A8180C612796A90094DF00E
:10762F00A3EFF090095012796D127A1C90094B124A
:10763F007A6190094D127A0D128B7F90094EE004FA
:10764F00F0700690094DE004F0127A7A7003127A06
:10765F0081C3900952E0941F900951E0940040CCEF
:10766F0012796A90094D127A1F900951E0FCA3E03C
:10767F00FDC3941FEC9400502290094D127A61AF14
:10768F00F0FE74A92DF582E43408F583E0FD128B2A
:10769F007F127A7A70D3127A8180CE1297D890099E
:1076AF004FE004F0A3E004F00275D79008A8E0FFC4
:1076BF0090094AE0FED39F5020900948E0FDA3E0D7
:1076CF00C39DFDE49400FCEE7A002DFDEA3CFCC363
:1076DF00ED9F7480F86C9850139008A8E0FF900904
:1076EF0048E0D39F500EA3E0C39F40089008A8E046
:0476FF00FF129A7864
:017703002263
:0389E00090095D9E
:1089E300127A2B129BEE90095EE0FE90095DE090F7
:1089F3000965127A88900961F090095FE0FF900998
:108A030065E0FCA3E0FD90099A1279B9741FF01296
:108A13009890900966E0241FF0900965E03400F017
:108A2300900961E0127A54A374FFF0A3EAF0A3E97A
:108A3300F0129BDF900962A3E0FAA3E0AE02FF907D
:108A430009A91279B9741FF01295481297D89009A1
:108A530061E004F0E0C3941E409F9008A8E0FF1279
:108A63009A789009E9E0FF129B7F900960E024FF68
:028A730092AFC0
:018A750022DE
:038C7B00900982DB
:108C7E00127A2B129BEE900983E0FE900982E0900F
:108C8E000987127A88900986F0900986E0FFC394CE
:108C9E001E504475F01FEF127971FE900989F0FA9B
:108CAE00A3EFF0FB900984E0FF900987E0FCA3E0BE
:108CBE00FDA9037BFF9009A2E4F0A3741FF01299A3
:108CCE00DF900988E0241FF0900987E03400F090CF
:108CDE000986E004F080B29009E9E0FF129B7F90D4
:078CEE000985E024FF92AFAD
:018CF500225C
:02889E00C119FE
:1083070090098BE025E024C9F582E43408F583223F
:10831700C3EF9BFFEE9AFEED9400FDEC9400FC90FA
:10832700099012443CE47F80FE900990FDFCE0F840
:10833700A3E0F9A3E0FAA3E0FBD30243BAF890095C
:108347008BE025E025E0246AF582E43407F58322F3
:1083570090098BE025E024A6F582E43407F5832213
:1083670074FF7F80FEFDFC900990E0F8A3A3A3E0D3
:10837700C30243BAE0FCA3E0FDA3E0FEA3E0FF12C3
:10838700429DE47BFF7A0FF9F822E0FEA3E0FFC3EA
:10839700EF9BFFEE9AFEE49400FDE49400FC227844
:1083A700041243F48E178F189009EAE0C41313548C
:1083B7000364022290098BE0245BF582E43407F51D
:1083C700832225E024E2F582E43407F58322E0C422
:1083D700F854F0C8682225E024C4F582E43407F590
:1083E700832290098CA3A3E0FEA3E022A3E0C45458
:0383F7000F48220A
:109A1300E4FFEF12830BE0FCA3E0FDEF1283C9EC3C
:099A2300F0A3EDF00FEFB40FE920
:019A2C002217
:0548360090098BEFF07A
:10483B009009EAE030E0179009D4E07004A3E0643B
:10484B0032600B90098BE0640B7003024B321283C6
:10485B0057E0FEA3E0FBAA06E490098BE075F01786
:10486B00A4241EF582E5F03404F58312839190099C
:10487B008C12443CE47FF47E0190098C128333400C
:10488B000E7516011283E9240CFFEE34FE80287F8F
:10489B000C7EFE7DFF7CFF90098CE0F8A3E0F9A372
:1048AB00E0FAA3E0FBC31243BA5018E4F5161283E7
:1048BB00E924F4FFEE3401FE128357EE8FF012421F
:1048CB007180071283BB7403F02290098BE0FD12F9
:1048DB00835B1283D5F5101283F3F511ED12830B65
:1048EB001283D5F5121283F3F51390098BE0128323
:1048FB00DD1283D5F5141283F3F515745B2D12833A
:10490B00C1E0B51603D38001C350030249D3E516AA
:02491B007039F1
:10491D00E5159401E514940050067E007F01800496
:10492D00AE14AF15E48F0B8E0AF509F508AE12AF74
:10493D00137C0F7DFF1244ABAB0BAA0AA909A80883
:06494D001243281283450D
:034953000249CA4C
:10495600AE14AF15AB07AA06C374FF9BF50F740F11
:104966009AF50EE49400F50DE49400F50CC374FF7B
:104976009513FF740F9512FE7C0F7DFF1244AB1248
:10498600834512443CE47F01FEFDFCAB0FAA0EA951
:104996000DA80CC31243D0500AE4750F01F50EF5AD
:1049A6000DF50C128345C083C082E0FCA3E0FDA395
:1049B600E0FEA3E0FFAB0FAA0EA90DA80C1293C24E
:0749C600D082D08312443CB3
:1049CD001283BBE516F0E516706FAE10AF11AB0795
:1049DD00AA06F912834412837B1293C21283A67026
:1049ED005590098BE0FF6406704C20190EEF128371
:1049FD000BE06517FEEE30E702D219201903024ACB
:014A0D00CCDC
:104A0E00128307E0FEA3E0FFE4FCFDC006C007AE84
:104A1E0017AF18AB07AA06D007D00612831750059A
:104A2E001283675003024ABD128307747FF0A3748A
:024A3E00FFF087
:104A4000024AD8024ACCAE10AF11AB07AA06C37413
:104A5000FF9BFB740F9AFAE49400F9E4940012832C
:104A60004412837B124328C374FF9FFF740F9EFE82
:104A7000E49DFDE49CFC1283A6705390098BE0FF3B
:104A80006406704A20190EEF12830BE06517FEEEE4
:084A900030E702D2193019349D
:104A9800128307E0FEA3E0FFE4FCFDC006C007AEFA
:104AA80017AF18AB07AA06D007D006128317500510
:104AB8001283675004C219800D1283077480F0A313
:024AC800E4F018
:104ACA00800C8000128307E517F0A3E518F090091F
:104ADA008BE0FF12835BE0FCA3E0FDEF1283DDECC9
:104AEA00F0A3EDF09009EAE030E003300706200079
:044AFA003720073426
:104AFE0090098BE01283C9E0FEA3E0FBAA061283A5
:104B0E000712839190099012443CE47F587E021262
:104B1E008330500D7FA87EFD7DFF7CFF12836E508B
:044B2E00031298B224
:014B32002260
:105036000000000100030004000600070009000A42
:10504600000C000E000F00110012001400150017CE
:105056000019001A001C001D001F00200022002459
:10506600002500270028002A002B002D002F0030E5
:1050760000320033003500360038003A003B003D70
:10508600003E0040004100430045004600480049FC
:10509600004B004C004E0050005100530054005687
:1050A60000570059005A005C005E005F0061006214
:1050B6000064006500670069006A006C006D006F9F
:1050C600007000720073007500770078007A007B2C
:1050D600007D007E008000820083008500860088B7
:1050E6000089008B008C008E009000910093009444
:1050F600009600970099009A009C009E009F00A1D0
:1051060000A200A400A500A700A800AA00AB00AD5D
:1051160000AF00B000B200B300B500B600B800B9E9
:1051260000BB00BC00BE00C000C100C300C400C676
:1051360000C700C900CA00CC00CD00CF00D100D204
:1051460000D400D500D700D800DA00DB00DD00DE91
:1051560000E000E100E300E400E600E800E900EB1F
:1051660000EC00EE00EF00F100F200F400F500F7AD
:1051760000F800FA00FB00FD00FE0100010101033A
:105186000104010601080109010B010C010E010FC2
:10519600011101120114011501170118011A011B51
:1051A600011D011E012001210123012401260127E1
:1051B6000129012A012C012D012F01300132013371
:1051C6000135013601380139013B013C013E013F01
:1051D600014101420144014501470148014A014B91
:1051E600014D014E01500151015301540156015721
:1051F6000158015A015B015D015E016001610163B5
:105206000164016601670169016A016C016D016F44
:105216000170017101730174017601770179017AD8
:10522600017C017D017F0180018201830184018669
:1052360001870189018A018C018D018F01900192FC
:1052460001930194019601970199019A019C019D90
:10525600019E01A001A101A301A401A601A701A825
:1052660001AA01AB01AD01AE01B001B101B201B4B9
:1052760001B501B701B801BA01BB01BC01BE01BF4E
:1052860001C101C201C301C501C601C801C901CAE4
:1052960001CC01CD01CF01D001D201D301D401D679
:1052A60001D701D801DA01DB01DD01DE01DF01E111
:1052B60001E201E401E501E601E801E901EB01ECA7
:1052C60001ED01EF01F001F101F301F401F501F740
:1052D60001F801FA01FB01FC01FE01FF02000202D6
:1052E60002030204020602070209020A020B020D69
:1052F600020E020F02110212021302150216021703
:105306000219021A021B021D021E021F022102229C
:1053160002230225022602270229022A022B022D37
:10532600022E022F023102320233023402360237D3
:105336000238023A023B023C023E023F024002426F
:10534600024302440245024702480249024B024C0C
:10535600024D024E025002510252025402550256AA
:1053660002570259025A025B025C025E025F026049
:105376000261026302640265026702680269026AE8
:10538600026C026D026E026F027102720273027487
:105396000275027702780279027A027C027D027E29
:1053A600027F0281028202830284028502870288CA
:1053B6000289028A028C028D028E028F029002926C
:1053C600029302940295029602980299029A029B0F
:1053D600029C029E029F02A002A102A202A302A5B3
:1053E60002A602A702A802A902AB02AC02AD02AE57
:1053F60002AF02B002B202B302B402B502B602B7FD
:1054060002B802BA02BB02BC02BD02BE02BF02C0A3
:1054160002C202C302C402C502C602C702C802CA49
:1054260002CB02CC02CD02CE02CF02D002D102D2F2
:1054360002D402D502D602D702D802D902DA02DB9A
:1054460002DC02DE02DF02E002E102E202E302E443
:1054560002E502E602E702E802E902EB02EC02EDEF
:1054660002EE02EF02F002F102F202F302F402F59A
:1054760002F602F702F802F902FA02FB02FD02FE48
:1054860002FF0300030103020303030403050306EB
:10549600030703080309030A030B030C030D030E9A
:1054A600030F03100311031203130314031503164A
:1054B600031703180319031A031B031C031D031EFA
:1054C600031F0320032103220323032403250326AA
:1054D600032703280329032A032B032C032D032D5B
:1054E600032E032F03300331033203330334033512
:1054F6000336033703380339033A033B033C033CC3
:10550600033D033E033F0340034103420343034479
:10551600034503460347034703480349034A034B2E
:10552600034C034D034E034F034F035003510352E5
:10553600035303540355035603560357035803599D
:10554600035A035B035C035C035D035E035F036056
:105556000361036103620363036403650366036611
:10556600036703680369036A036B036B036C036DCC
:10557600036E036F036F0370037103720373037388
:105586000374037503760377037703780379037A45
:10559600037A037B037C037D037E037E037F038004
:1055A60003810381038203830384038403850386C3
:1055B6000387038703880389038A038A038B038C83
:1055C600038C038D038E038F038F03900391039146
:1055D6000392039303940394039503960396039708
:1055E600039803980399039A039A039B039C039DCC
:1055F600039D039E039F039F03A003A103A103A290
:1056060003A203A303A403A403A503A603A603A757
:1056160003A803A803A903AA03AA03AB03AB03AC1D
:1056260003AD03AD03AE03AF03AF03B003B003B1E5
:1056360003B203B203B303B303B403B503B503B6AE
:1056460003B603B703B703B803B903B903BA03BA7A
:1056560003BB03BB03BC03BD03BD03BE03BE03BF45
:1056660003BF03C003C003C103C203C203C303C312
:1056760003C403C403C503C503C603C603C703C7E0
:1056860003C803C803C903C903CA03CA03CB03CBB0
:1056960003CC03CC03CD03CD03CE03CE03CF03CF80
:1056A60003D003D003D103D103D203D203D203D351
:1056B60003D303D403D403D503D503D603D603D724
:1056C60003D703D703D803D803D903D903DA03DAF8
:1056D60003DA03DB03DB03DC03DC03DC03DD03DDCE
:1056E60003DE03DE03DE03DF03DF03E003E003E0A4
:1056F60003E103E103E203E203E203E303E303E37B
:1057060003E403E403E503E503E503E603E603E652
:1057160003E703E703E703E803E803E803E903E92C
:1057260003E903EA03EA03EA03EB03EB03EB03EC07
:1057360003EC03EC03EC03ED03ED03ED03EE03EEE4
:1057460003EE03EE03EF03EF03EF03F003F003F0C2
:1057560003F003F103F103F103F103F203F203F2A1
:1057660003F203F303F303F303F303F403F403F481
:1057760003F403F503F503F503F503F603F603F661
:1057860003F603F603F703F703F703F703F703F844
:1057960003F803F803F803F803F903F903F903F927
:1057A60003F903F903FA03FA03FA03FA03FA03FA0D
:1057B60003FB03FB03FB03FB03FB03FB03FB03FCF2
:1057C60003FC03FC03FC03FC03FC03FC03FC03FDDA
:1057D60003FD03FD03FD03FD03FD03FD03FD03FDC3
:1057E60003FE03FE03FE03FE03FE03FE03FE03FEAB
:1057F60003FE03FE03FE03FE03FF03FF03FF03FF97
:1058060003FF03FF03FF03FF03FF03FF03FF03FF82
:1058160003FF03FF03FF03FF03FF03FF03FF03FF72
:1058260003FF03FF03FF03FF03FF03FF03FF03FF62
:1058360003FF03FF03FF03FF03FF03FF03FF03FF52
:1058460003FF03FF03FF03FF03FF03FF03FF03FF42
:1058560003FF03FF03FF03FF03FF03FF03FF03FF32
:1058660003FF03FF03FF03FF03FF03FE03FE03FE25
:1058760003FE03FE03FE03FE03FE03FE03FE03FE1A
:1058860003FE03FD03FD03FD03FD03FD03FD03FD11
:1058960003FD03FD03FC03FC03FC03FC03FC03FC08
:1058A60003FC03FC03FB03FB03FB03FB03FB03FB00
:1058B60003FB03FA03FA03FA03FA03FA03FA03F9FA
:1058C60003F903F903F903F903F903F803F803F8F5
:1058D60003F803F803F703F703F703F703F703F6F1
:1058E60003F603F603F603F603F503F503F503F5EE
:1058F60003F403F403F403F403F303F303F303F3EE
:1059060003F203F203F203F203F103F103F103F1ED
:1059160003F003F003F003F003EF03EF03EF03EEEE
:1059260003EE03EE03EE03ED03ED03ED03EC03ECF0
:1059360003EC03EC03EB03EB03EB03EA03EA03EAF2
:1059460003E903E903E903E803E803E803E703E7F8
:1059560003E703E603E603E603E503E503E503E4FD
:1059660003E403E303E303E303E203E203E203E105
:1059760003E103E003E003E003DF03DF03DE03DE0E
:1059860003DE03DD03DD03DC03DC03DC03DB03DB17
:1059960003DA03DA03DA03D903D903D803D803D722
:1059A60003D703D703D603D603D503D503D403D42D
:1059B60003D303D303D203D203D203D103D103D03B
:1059C60003D003CF03CF03CE03CE03CD03CD03CC49
:1059D60003CC03CB03CB03CA03CA03C903C903C859
:1059E60003C803C703C703C603C603C503C503C469
:1059F60003C403C303C303C203C203C103C003C07A
:105A060003BF03BF03BE03BE03BD03BD03BC03BB8D
:105A160003BB03BA03BA03B903B903B803B703B7A1
:105A260003B603B603B503B503B403B303B303B2B6
:105A360003B203B103B003B003AF03AF03AE03ADCC
:105A460003AD03AC03AB03AB03AA03AA03A903A8E4
:105A560003A803A703A603A603A503A403A403A3FD
:105A660003A203A203A103A103A0039F039F039E16
:105A7600039D039D039C039B039A039A0399039832
:105A8600039803970396039603950394039403934D
:105A96000392039103910390038F038F038E038D6B
:105AA600038C038C038B038A038A03890388038789
:105AB60003870386038503840384038303820381A8
:105AC60003810380037F037E037E037D037C037BC8
:105AD600037A037A037903780377037703760375EA
:105AE600037403730373037203710370036F036F0D
:105AF600036E036D036C036B036B036A0369036830
:105B06000367036603660365036403630362036155
:105B160003610360035F035E035D035C035C035B79
:105B2600035A0359035803570356035603550354A0
:105B36000353035203510350034F034F034E034DC8
:105B4600034C034B034A03490348034703470346F1
:105B5600034503440343034203410340033F033E1B
:105B6600033D033C033C033B033A03390338033745
:105B76000336033503340333033203310330032F73
:105B8600032E032D032D032C032B032A032903289D
:105B960003270326032503240323032203210320CB
:105BA600031F031E031D031C031B031A03190318FB
:105BB600031703160315031403130312031103102B
:105BC600030F030E030D030C030B030A030903085B
:105BD600030703060305030403030302030103008B
:105BE60002FF02FE02FD02FB02FA02F902F802F7C8
:105BF60002F602F502F402F302F202F102F002EFFB
:105C060002EE02ED02EC02EB02E902E802E702E62E
:105C160002E502E402E302E202E102E002DF02DE62
:105C260002DC02DB02DA02D902D802D702D602D59A
:105C360002D402D202D102D002CF02CE02CD02CCD1
:105C460002CB02CA02C802C702C602C502C402C308
:105C560002C202C002BF02BE02BD02BC02BB02BA41
:105C660002B802B702B602B502B402B302B102B07C
:105C760002AF02AE02AD02AC02AB02A902A802A7B5
:105C860002A602A502A302A202A102A0029F029EF0
:105C9600029C029B029A029902980296029502942D
:105CA600029302920290028F028E028D028C028A69
:105CB60002890288028702850284028302820281A7
:105CC600027F027E027D027C027A027902780277E6
:105CD60002750274027302720271026F026E026D25
:105CE600026C026A02690268026702650264026364
:105CF60002610260025F025E025C025B025A0259A6
:105D06000257025602550254025202510250024EE6
:105D1600024D024C024B0249024802470245024428
:105D2600024302420240023F023E023C023B023A6A
:105D36000238023702360234023302320231022FAF
:105D4600022E022D022B022A0229022702260225F2
:105D5600022302220221021F021E021D021B021A38
:105D66000219021702160215021302120211020F7D
:105D7600020E020D020B020A0209020702060204C3
:105D860002030202020001FF01FE01FC01FB01FA0F
:105D960001F801F701F501F401F301F101F001EF5A
:105DA60001ED01EC01EA01E901E801E601E501E4A2
:105DB60001E201E101DF01DE01DD01DB01DA01D8EB
:105DC60001D701D601D401D301D201D001CF01CD33
:105DD60001CC01CA01C901C801C601C501C301C27E
:105DE60001C101BF01BE01BC01BB01BA01B801B7C7
:105DF60001B501B401B201B101B001AE01AD01AB13
:105E060001AA01A801A701A601A401A301A101A05D
:105E1600019E019D019C019A0199019701960194A9
:105E2600019301920190018F018D018C018A0189F4
:105E3600018701860184018301820180017F017D42
:105E4600017C017A01790177017601740173017190
:105E56000170016F016D016C016A016901670166DC
:105E66000164016301610160015E015D015B015A2C
:105E76000158015701560154015301510150014E79
:105E8600014D014B014A01480147014501440142C8
:105E96000141013F013E013C013B01390138013618
:105EA6000135013301320130012F012D012C012A68
:105EB6000129012701260124012301210120011EB8
:105EC600011D011B011A0118011701150114011208
:105ED6000111010F010E010C010B01090108010658
:105EE600010401030101010000FE00FD00FB00FAB0
:105EF60000F800F700F500F400F200F100EF00EE04
:105F060000EC00EB00E900E800E600E400E300E155
:105F160000E000DE00DD00DB00DA00D800D700D5A7
:105F260000D400D200D100CF00CD00CC00CA00C9F9
:105F360000C700C600C400C300C100C000BE00BC4C
:105F460000BB00B900B800B600B500B300B200B09F
:105F560000AF00AD00AB00AA00A800A700A500A4F2
:105F660000A200A1009F009E009C009A0099009745
:105F760000960094009300910090008E008C008B98
:105F86000089008800860085008300820080007EEC
:105F9600007D007B007A0078007700750073007240
:105FA6000070006F006D006C006A00690067006594
:105FB600006400620061005F005E005C005A0059E8
:105FC600005700560054005300510050004E004C3C
:105FD600004B004900480046004500430041004090
:105FE600003E003D003B003A0038003600350033E5
:105FF60000320030002F002D002B002A0028002739
:106006000025002400220020001F001D001C001A8D
:10601600001900170015001400120011000F000EE1
:10602600000C000A00090007000600040003000136
:106036000000FFFFFFFDFFFCFFFAFFF9FFF7FFF689
:10604600FFF4FFF2FFF1FFEFFFEEFFECFFEBFFE9DE
:10605600FFE7FFE6FFE4FFE3FFE1FFE0FFDEFFDC33
:10606600FFDBFFD9FFD8FFD6FFD5FFD3FFD1FFD087
:10607600FFCEFFCDFFCBFFCAFFC8FFC6FFC5FFC3DC
:10608600FFC2FFC0FFBFFFBDFFBBFFBAFFB8FFB730
:10609600FFB5FFB4FFB2FFB0FFAFFFADFFACFFAA85
:1060A600FFA9FFA7FFA6FFA4FFA2FFA1FF9FFF9ED8
:1060B600FF9CFF9BFF99FF97FF96FF94FF93FF912D
:1060C600FF90FF8EFF8DFF8BFF89FF88FF86FF8580
:1060D600FF83FF82FF80FF7EFF7DFF7BFF7AFF78D5
:1060E600FF77FF75FF74FF72FF70FF6FFF6DFF6C28
:1060F600FF6AFF69FF67FF66FF64FF62FF61FF5F7C
:10610600FF5EFF5CFF5BFF59FF58FF56FF55FF53CD
:10611600FF51FF50FF4EFF4DFF4BFF4AFF48FF4721
:10612600FF45FF44FF42FF40FF3FFF3DFF3CFF3A74
:10613600FF39FF37FF36FF34FF33FF31FF2FFF2EC6
:10614600FF2CFF2BFF29FF28FF26FF25FF23FF2219
:10615600FF20FF1FFF1DFF1CFF1AFF18FF17FF156B
:10616600FF14FF12FF11FF0FFF0EFF0CFF0BFF09BD
:10617600FF08FF06FF05FF03FF02FF00FEFFFEFD0F
:10618600FEFCFEFAFEF8FEF7FEF5FEF4FEF2FEF168
:10619600FEEFFEEEFEECFEEBFEE9FEE8FEE6FEE5B9
:1061A600FEE3FEE2FEE0FEDFFEDDFEDCFEDAFED909
:1061B600FED7FED6FED4FED3FED1FED0FECEFECD59
:1061C600FECBFECAFEC8FEC7FEC5FEC4FEC2FEC1A9
:1061D600FEBFFEBEFEBCFEBBFEB9FEB8FEB6FEB5F9
:1061E600FEB3FEB2FEB0FEAFFEADFEACFEAAFEA949
:1061F600FEA8FEA6FEA5FEA3FEA2FEA0FE9FFE9D95
:10620600FE9CFE9AFE99FE97FE96FE94FE93FE91E4
:10621600FE90FE8EFE8DFE8CFE8AFE89FE87FE8631
:10622600FE84FE83FE81FE80FE7EFE7DFE7CFE7A7F
:10623600FE79FE77FE76FE74FE73FE71FE70FE6ECC
:10624600FE6DFE6CFE6AFE69FE67FE66FE64FE6318
:10625600FE62FE60FE5FFE5DFE5CFE5AFE59FE5863
:10626600FE56FE55FE53FE52FE50FE4FFE4EFE4CAF
:10627600FE4BFE49FE48FE46FE45FE44FE42FE41FA
:10628600FE3FFE3EFE3DFE3BFE3AFE38FE37FE3545
:10629600FE34FE33FE31FE30FE2EFE2DFE2CFE2A8F
:1062A600FE29FE28FE26FE25FE23FE22FE21FE1FD7
:1062B600FE1EFE1CFE1BFE1AFE18FE17FE15FE1421
:1062C600FE13FE11FE10FE0FFE0DFE0CFE0BFE0968
:1062D600FE08FE06FE05FE04FE02FE01FE00FDFEB1
:1062E600FDFDFDFCFDFAFDF9FDF7FDF6FDF5FDF3FF
:1062F600FDF2FDF1FDEFFDEEFDEDFDEBFDEAFDE945
:10630600FDE7FDE6FDE5FDE3FDE2FDE1FDDFFDDE8A
:10631600FDDDFDDBFDDAFDD9FDD7FDD6FDD5FDD3CF
:10632600FDD2FDD1FDCFFDCEFDCDFDCCFDCAFDC913
:10633600FDC8FDC6FDC5FDC4FDC2FDC1FDC0FDBE57
:10634600FDBDFDBCFDBBFDB9FDB8FDB7FDB5FDB49A
:10635600FDB3FDB2FDB0FDAFFDAEFDACFDABFDAADC
:10636600FDA9FDA7FDA6FDA5FDA4FDA2FDA1FDA01D
:10637600FD9FFD9DFD9CFD9BFD99FD98FD97FD965E
:10638600FD94FD93FD92FD91FD8FFD8EFD8DFD8C9F
:10639600FD8AFD89FD88FD87FD86FD84FD83FD82DE
:1063A600FD81FD7FFD7EFD7DFD7CFD7BFD79FD781C
:1063B600FD77FD76FD74FD73FD72FD71FD70FD6E5A
:1063C600FD6DFD6CFD6BFD6AFD68FD67FD66FD6597
:1063D600FD64FD62FD61FD60FD5FFD5EFD5DFD5BD3
:1063E600FD5AFD59FD58FD57FD55FD54FD53FD520F
:1063F600FD51FD50FD4EFD4DFD4CFD4BFD4AFD4949
:10640600FD48FD46FD45FD44FD43FD42FD41FD4081
:10641600FD3EFD3DFD3CFD3BFD3AFD39FD38FD36BB
:10642600FD35FD34FD33FD32FD31FD30FD2FFD2EF2
:10643600FD2CFD2BFD2AFD29FD28FD27FD26FD252A
:10644600FD24FD22FD21FD20FD1FFD1EFD1DFD1C61
:10645600FD1BFD1AFD19FD18FD17FD15FD14FD1395
:10646600FD12FD11FD10FD0FFD0EFD0DFD0CFD0BCA
:10647600FD0AFD09FD08FD07FD06FD05FD03FD02FC
:10648600FD01FD00FCFFFCFEFCFDFCFCFCFBFCFA38
:10649600FCF9FCF8FCF7FCF6FCF5FCF4FCF3FCF26A
:1064A600FCF1FCF0FCEFFCEEFCEDFCECFCEBFCEA9A
:1064B600FCE9FCE8FCE7FCE6FCE5FCE4FCE3FCE2CA
:1064C600FCE1FCE0FCDFFCDEFCDDFCDCFCDBFCDAFA
:1064D600FCD9FCD8FCD7FCD6FCD5FCD4FCD3FCD329
:1064E600FCD2FCD1FCD0FCCFFCCEFCCDFCCCFCCB52
:1064F600FCCAFCC9FCC8FCC7FCC6FCC5FCC4FCC481
:10650600FCC3FCC2FCC1FCC0FCBFFCBEFCBDFCBCA9
:10651600FCBBFCBAFCB9FCB9FCB8FCB7FCB6FCB5D4
:10652600FCB4FCB3FCB2FCB1FCB1FCB0FCAFFCAEFD
:10653600FCADFCACFCABFCAAFCAAFCA9FCA8FCA725
:10654600FCA6FCA5FCA4FCA4FCA3FCA2FCA1FCA04C
:10655600FC9FFC9FFC9EFC9DFC9CFC9BFC9AFC9A71
:10656600FC99FC98FC97FC96FC95FC95FC94FC9396
:10657600FC92FC91FC91FC90FC8FFC8EFC8DFC8DBA
:10658600FC8CFC8BFC8AFC89FC89FC88FC87FC86DD
:10659600FC86FC85FC84FC83FC82FC82FC81FC80FE
:1065A600FC7FFC7FFC7EFC7DFC7CFC7CFC7BFC7A1F
:1065B600FC79FC79FC78FC77FC76FC76FC75FC743F
:1065C600FC74FC73FC72FC71FC71FC70FC6FFC6F5C
:1065D600FC6EFC6DFC6CFC6CFC6BFC6AFC6AFC697A
:1065E600FC68FC68FC67FC66FC66FC65FC64FC6396
:1065F600FC63FC62FC61FC61FC60FC5FFC5FFC5EB2
:10660600FC5EFC5DFC5CFC5CFC5BFC5AFC5AFC59C9
:10661600FC58FC58FC57FC56FC56FC55FC55FC54E3
:10662600FC53FC53FC52FC51FC51FC50FC50FC4FFB
:10663600FC4EFC4EFC4DFC4DFC4CFC4BFC4BFC4A12
:10664600FC4AFC49FC49FC48FC47FC47FC46FC4626
:10665600FC45FC45FC44FC43FC43FC42FC42FC413B
:10666600FC41FC40FC40FC3FFC3EFC3EFC3DFC3D4E
:10667600FC3CFC3CFC3BFC3BFC3AFC3AFC39FC3960
:10668600FC38FC38FC37FC37FC36FC36FC35FC3570
:10669600FC34FC34FC33FC33FC32FC32FC31FC3180
:1066A600FC30FC30FC2FFC2FFC2EFC2EFC2EFC2D8F
:1066B600FC2DFC2CFC2CFC2BFC2BFC2AFC2AFC299C
:1066C600FC29FC29FC28FC28FC27FC27FC26FC26A8
:1066D600FC26FC25FC25FC24FC24FC24FC23FC23B2
:1066E600FC22FC22FC22FC21FC21FC20FC20FC20BC
:1066F600FC1FFC1FFC1EFC1EFC1EFC1DFC1DFC1DC5
:10670600FC1CFC1CFC1BFC1BFC1BFC1AFC1AFC1ACC
:10671600FC19FC19FC19FC18FC18FC18FC17FC17D2
:10672600FC17FC16FC16FC16FC15FC15FC15FC14D7
:10673600FC14FC14FC14FC13FC13FC13FC12FC12DA
:10674600FC12FC12FC11FC11FC11FC10FC10FC10DC
:10675600FC10FC0FFC0FFC0FFC0FFC0EFC0EFC0EDD
:10676600FC0EFC0DFC0DFC0DFC0DFC0CFC0CFC0CDD
:10677600FC0CFC0BFC0BFC0BFC0BFC0AFC0AFC0ADD
:10678600FC0AFC0AFC09FC09FC09FC09FC09FC08DA
:10679600FC08FC08FC08FC08FC07FC07FC07FC07D7
:1067A600FC07FC07FC06FC06FC06FC06FC06FC06D1
:1067B600FC05FC05FC05FC05FC05FC05FC05FC04CC
:1067C600FC04FC04FC04FC04FC04FC04FC04FC03C4
:1067D600FC03FC03FC03FC03FC03FC03FC03FC03BB
:1067E600FC02FC02FC02FC02FC02FC02FC02FC02B3
:1067F600FC02FC02FC02FC02FC01FC01FC01FC01A7
:10680600FC01FC01FC01FC01FC01FC01FC01FC019A
:10681600FC01FC01FC01FC01FC01FC01FC01FC018A
:10682600FC01FC01FC01FC01FC01FC01FC01FC017A
:10683600FC01FC01FC01FC01FC01FC01FC01FC016A
:10684600FC01FC01FC01FC01FC01FC01FC01FC015A
:10685600FC01FC01FC01FC01FC01FC01FC01FC014A
:10686600FC01FC01FC01FC01FC01FC02FC02FC0237
:10687600FC02FC02FC02FC02FC02FC02FC02FC0222
:10688600FC02FC03FC03FC03FC03FC03FC03FC030B
:10689600FC03FC03FC04FC04FC04FC04FC04FC04F4
:1068A600FC04FC04FC05FC05FC05FC05FC05FC05DC
:1068B600FC05FC06FC06FC06FC06FC06FC06FC07C2
:1068C600FC07FC07FC07FC07FC07FC08FC08FC08A7
:1068D600FC08FC08FC09FC09FC09FC09FC09FC0A8B
:1068E600FC0AFC0AFC0AFC0AFC0BFC0BFC0BFC0B6E
:1068F600FC0CFC0CFC0CFC0CFC0DFC0DFC0DFC0D4E
:10690600FC0EFC0EFC0EFC0EFC0FFC0FFC0FFC0F2D
:10691600FC10FC10FC10FC10FC11FC11FC11FC120C
:10692600FC12FC12FC12FC13FC13FC13FC14FC14EA
:10693600FC14FC14FC15FC15FC15FC16FC16FC16C8
:10694600FC17FC17FC17FC18FC18FC18FC19FC19A2
:10695600FC19FC1AFC1AFC1AFC1BFC1BFC1BFC1C7D
:10696600FC1CFC1DFC1DFC1DFC1EFC1EFC1EFC1F55
:10697600FC1FFC20FC20FC20FC21FC21FC22FC222C
:10698600FC22FC23FC23FC24FC24FC24FC25FC2503
:10699600FC26FC26FC26FC27FC27FC28FC28FC29D8
:1069A600FC29FC29FC2AFC2AFC2BFC2BFC2CFC2CAD
:1069B600FC2DFC2DFC2EFC2EFC2EFC2FFC2FFC307F
:1069C600FC30FC31FC31FC32FC32FC33FC33FC3451
:1069D600FC34FC35FC35FC36FC36FC37FC37FC3821
:1069E600FC38FC39FC39FC3AFC3AFC3BFC3BFC3CF1
:1069F600FC3CFC3DFC3DFC3EFC3EFC3FFC40FC40C0
:106A0600FC41FC41FC42FC42FC43FC43FC44FC458B
:106A1600FC45FC46FC46FC47FC47FC48FC49FC4957
:106A2600FC4AFC4AFC4BFC4BFC4CFC4DFC4DFC4E22
:106A3600FC4EFC4FFC50FC50FC51FC51FC52FC53EC
:106A4600FC53FC54FC55FC55FC56FC56FC57FC58B4
:106A5600FC58FC59FC5AFC5AFC5BFC5CFC5CFC5D7B
:106A6600FC5EFC5EFC5FFC5FFC60FC61FC61FC6242
:106A7600FC63FC63FC64FC65FC66FC66FC67FC6806
:106A8600FC68FC69FC6AFC6AFC6BFC6CFC6CFC6DCB
:106A9600FC6EFC6FFC6FFC70FC71FC71FC72FC738D
:106AA600FC74FC74FC75FC76FC76FC77FC78FC794F
:106AB600FC79FC7AFC7BFC7CFC7CFC7DFC7EFC7F10
:106AC600FC7FFC80FC81FC82FC82FC83FC84FC85D0
:106AD600FC86FC86FC87FC88FC89FC89FC8AFC8B8E
:106AE600FC8CFC8DFC8DFC8EFC8FFC90FC91FC914B
:106AF600FC92FC93FC94FC95FC95FC96FC97FC9808
:106B0600FC99FC9AFC9AFC9BFC9CFC9DFC9EFC9FC1
:106B1600FC9FFCA0FCA1FCA2FCA3FCA4FCA4FCA57D
:106B2600FCA6FCA7FCA8FCA9FCAAFCAAFCABFCAC36
:106B3600FCADFCAEFCAFFCB0FCB1FCB1FCB2FCB3EE
:106B4600FCB4FCB5FCB6FCB7FCB8FCB9FCB9FCBAA5
:106B5600FCBBFCBCFCBDFCBEFCBFFCC0FCC1FCC25B
:106B6600FCC3FCC4FCC4FCC5FCC6FCC7FCC8FCC911
:106B7600FCCAFCCBFCCCFCCDFCCEFCCFFCD0FCD1C3
:106B8600FCD2FCD3FCD3FCD4FCD5FCD6FCD7FCD879
:106B9600FCD9FCDAFCDBFCDCFCDDFCDEFCDFFCE02B
:106BA600FCE1FCE2FCE3FCE4FCE5FCE6FCE7FCE8DB
:106BB600FCE9FCEAFCEBFCECFCEDFCEEFCEFFCF08B
:106BC600FCF1FCF2FCF3FCF4FCF5FCF6FCF7FCF83B
:106BD600FCF9FCFAFCFBFCFCFCFDFCFEFCFFFD00EA
:106BE600FD01FD02FD03FD05FD06FD07FD08FD098E
:106BF600FD0AFD0BFD0CFD0DFD0EFD0FFD10FD113B
:106C0600FD12FD13FD14FD15FD17FD18FD19FD1AE6
:106C1600FD1BFD1CFD1DFD1EFD1FFD20FD21FD2292
:106C2600FD24FD25FD26FD27FD28FD29FD2AFD2B3A
:106C3600FD2CFD2EFD2FFD30FD31FD32FD33FD34E3
:106C4600FD35FD36FD38FD39FD3AFD3BFD3CFD3D8C
:106C5600FD3EFD40FD41FD42FD43FD44FD45FD4633
:106C6600FD48FD49FD4AFD4BFD4CFD4DFD4FFD50D8
:106C7600FD51FD52FD53FD54FD55FD57FD58FD597F
:106C8600FD5AFD5BFD5DFD5EFD5FFD60FD61FD6224
:106C9600FD64FD65FD66FD67FD68FD6AFD6BFD6CC7
:106CA600FD6DFD6EFD70FD71FD72FD73FD74FD766B
:106CB600FD77FD78FD79FD7BFD7CFD7DFD7EFD7F0D
:106CC600FD81FD82FD83FD84FD86FD87FD88FD89AE
:106CD600FD8BFD8CFD8DFD8EFD8FFD91FD92FD934F
:106CE600FD94FD96FD97FD98FD99FD9BFD9CFD9DF0
:106CF600FD9FFDA0FDA1FDA2FDA4FDA5FDA6FDA78E
:106D0600FDA9FDAAFDABFDACFDAEFDAFFDB0FDB22C
:106D1600FDB3FDB4FDB5FDB7FDB8FDB9FDBBFDBCCA
:106D2600FDBDFDBEFDC0FDC1FDC2FDC4FDC5FDC668
:106D3600FDC8FDC9FDCAFDCCFDCDFDCEFDCFFDD103
:106D4600FDD2FDD3FDD5FDD6FDD7FDD9FDDAFDDBA0
:106D5600FDDDFDDEFDDFFDE1FDE2FDE3FDE5FDE63A
:106D6600FDE7FDE9FDEAFDEBFDEDFDEEFDEFFDF1D5
:106D7600FDF2FDF3FDF5FDF6FDF7FDF9FDFAFDFC6F
:106D8600FDFDFDFEFE00FE01FE02FE04FE05FE0602
:106D9600FE08FE09FE0BFE0CFE0DFE0FFE10FE1198
:106DA600FE13FE14FE16FE17FE18FE1AFE1BFE1C30
:106DB600FE1EFE1FFE21FE22FE23FE25FE26FE28C7
:106DC600FE29FE2AFE2CFE2DFE2FFE30FE31FE335E
:106DD600FE34FE36FE37FE38FE3AFE3BFE3DFE3EF4
:106DE600FE3FFE41FE42FE44FE45FE46FE48FE498B
:106DF600FE4BFE4CFE4EFE4FFE50FE52FE53FE551F
:106E0600FE56FE58FE59FE5AFE5CFE5DFE5FFE60B3
:106E1600FE62FE63FE64FE66FE67FE69FE6AFE6C47
:106E2600FE6DFE6FFE70FE71FE73FE74FE76FE77DB
:106E3600FE79FE7AFE7CFE7DFE7EFE80FE81FE836E
:106E4600FE84FE86FE87FE89FE8AFE8CFE8DFE8F00
:106E5600FE90FE91FE93FE94FE96FE97FE99FE9A94
:106E6600FE9CFE9DFE9FFEA0FEA2FEA3FEA5FEA624
:106E7600FEA8FEA9FEAAFEACFEADFEAFFEB0FEB2B7
:106E8600FEB3FEB5FEB6FEB8FEB9FEBBFEBCFEBE48
:106E9600FEBFFEC1FEC2FEC4FEC5FEC7FEC8FECAD8
:106EA600FECBFECDFECEFED0FED1FED3FED4FED668
:106EB600FED7FED9FEDAFEDCFEDDFEDFFEE0FEE2F8
:106EC600FEE3FEE5FEE6FEE8FEE9FEEBFEECFEEE88
:106ED600FEEFFEF1FEF2FEF4FEF5FEF7FEF8FEFA18
:106EE600FEFCFEFDFEFFFF00FF02FF03FF05FF069F
:106EF600FF08FF09FF0BFF0CFF0EFF0FFF11FF122C
:106F0600FF14FF15FF17FF18FF1AFF1CFF1DFF1FB9
:106F1600FF20FF22FF23FF25FF26FF28FF29FF2B47
:106F2600FF2CFF2EFF2FFF31FF33FF34FF36FF37D5
:106F3600FF39FF3AFF3CFF3DFF3FFF40FF42FF4462
:106F4600FF45FF47FF48FF4AFF4BFF4DFF4EFF50EF
:106F5600FF51FF53FF55FF56FF58FF59FF5BFF5C7C
:106F6600FF5EFF5FFF61FF62FF64FF66FF67FF6909
:106F7600FF6AFF6CFF6DFF6FFF70FF72FF74FF7596
:106F8600FF77FF78FF7AFF7BFF7DFF7EFF80FF8222
:106F9600FF83FF85FF86FF88FF89FF8BFF8DFF8EAE
:106FA600FF90FF91FF93FF94FF96FF97FF99FF9B3A
:106FB600FF9CFF9EFF9FFFA1FFA2FFA4FFA6FFA7C6
:106FC600FFA9FFAAFFACFFADFFAFFFB0FFB2FFB452
:106FD600FFB5FFB7FFB8FFBAFFBBFFBDFFBFFFC0DE
:106FE600FFC2FFC3FFC5FFC6FFC8FFCAFFCBFFCD69
:106FF600FFCEFFD0FFD1FFD3FFD5FFD6FFD8FFD9F5
:10700600FFDBFFDCFFDEFFE0FFE1FFE3FFE4FFE67F
:10701600FFE7FFE9FFEBFFECFFEEFFEFFFF1FFF20B
:10702600FFF4FFF6FFF7FFF9FFFAFFFCFFFDFFFF96
:03000000024000BB
:03000300025003A5
:03000B000250069A
:030013000250098F
:03001B0002500C84
:0300230002500F79
:03002B000250126E
:0300330002501563
:03003B0002501858
:0300430002501B4D
:03004B0002501E42
:0300530002502137
:03005B000250242C
:0300630002502721
:03006B0002502A16
:0300730002502D0B
:03007B0002503000
:03008300025033F5
:03008B00025036EA
:03009300025039DF
:03009B0002503CD4
:0300A30002503FC9
:10400000787FE4F6D8FD9000007F007E20E4F0A3E6
:0A401000DFFCDEFA758169024055FD
:10401A00024504E493A3F8E493A34003F68001F273
:10402A0008DFF48029E493A3F85407240CC8C333A7
:10403A00C4540F4420C8834004F456800146F6DF76
:10404A00E4800B01020408102040809087EAE47E95
:10405A00019360BCA3FF543F30E509541FFEE4936B
:10406A00A360010ECF54C025E060A840B8E493A332
:10407A00FAE493A3F8E493A3C8C582C8CAC583CA5D
:10408A00F0A3C8C582C8CAC583CADFE9DEE780BE15
:0188A00000D7
:10409A00E709F608DFFA8046E709F208DFFA803E08
:1040AA0088828C83E709F0A3DFFA8032E309F608F5
:1040BA00DFFA8078E309F208DFFA807088828C835D
:1040CA00E309F0A3DFFA806489828A83E0A3F60811
:1040DA00DFFA805889828A83E0A3F208DFFA804CEB
:1040EA0080D280FA80C680D4806980F280338010C2
:1040FA0080A680EA809A80A880DA80E280CA80332B
:10410A0089828A83ECFAE493A3C8C582C8CCC583A2
:10411A00CCF0A3C8C582C8CCC583CCDFE9DEE78072
:10412A000D89828A83E493A3F608DFF9ECFAA9F0F1
:10413A00EDFB2289828A83ECFAE0A3C8C582C8CC47
:10414A00C583CCF0A3C8C582C8CCC583CCDFEADE60
:10415A00E880DB89828A83E493A3F208DFF980CCC2
:10416A0088F0EF60010E4E60C388F0ED2402B404BB
:10417A000050B9F582EB2402B4040050AF23234562
:06418A0082239040EA735D
:10419000BB010689828A83E0225002E722BBFE022D
:0941A000E32289828A83E4932260
:1041A900BB010CE58229F582E5833AF583E02250CB
:1041B90006E92582F8E622BBFE06E92582F8E22215
:0D41C900E58229F582E5833AF583E493222F
:1041D600BB010689828A83F0225002F722BBFE01C8
:0241E600F322C2
:1041E800F8BB010DE58229F582E5833AF583E8F00D
:1041F800225006E92582C8F622BBFE05E92582C8B9
:02420800F222A0
:10420A00EF8DF0A4A8F0CF8CF0A428CE8DF0A42EC8
:02421A00FE2282
:10421C00BC000BBE0029EF8DF084FFADF022E4CC86
:10422C00F875F008EF2FFFEE33FEEC33FCEE9DEC4F
:10423C00984005FCEE9DFE0FD5F0E9E4CEFD22ED95
:10424C00F8F5F0EE8420D21CFEADF075F008EF2FDF
:10425C00FFED33FD4007985006D5F0F222C398FDD0
:05426C000FD5F0EA226D
:10427100C5F0F8A3E028F0C5F0F8E58215827002D8
:064281001583E038F02275
:10428700A3F8E0C5F025F0F0E582158270021583EA
:06429700E0C838F0E82247
:10429D00E88FF0A4CC8BF0A42CFCE98EF0A42CFCC0
:1042AD008AF0EDA42CFCEA8EF0A4CDA8F08BF0A43E
:1042BD002DCC3825F0FDE98FF0A42CCD35F0FCEB9D
:1042CD008EF0A4FEA9F0EB8FF0A4CFC5F02ECD3962
:0F42DD00FEE43CFCEAA42DCE35F0FDE43CFC22CF
:1042EC0075F008758200EF2FFFEE33FECD33CDCC89
:1042FC0033CCC58233C5829BED9AEC99E58298400C
:10430C000CF582EE9BFEED9AFDEC99FC0FD5F0D6E8
:10431C00E4CEFBE4CDFAE4CCF9A88222B800C1B912
:10432C000059BA002DEC8BF084CFCECDFCE5F0CB50
:10433C00F97818EF2FFFEE33FEED33FDEC33FCEB89
:10434C0033FB10D703994004EB99FB0FD8E5E4F944
:10435C00FA227818EF2FFFEE33FEED33FDEC33FC31
:10436C00C933C910D7059BE99A4007EC9BFCE99A25
:10437C00F90FD8E0E4C9FAE4CCFB2275F010EF2F6A
:10438C00FFEE33FEED33FDCC33CCC833C810D7076A
:10439C009BEC9AE899400AED9BFDEC9AFCE899F8A5
:0E43AC000FD5F0DAE4CDFBE4CCFAE4C8F92238
:1093C200C2D5E830E70FB2D5E4C39BFBE49AFAE4D6
:1093D20099F9E498F8EC30E717B2D51293F81243F2
:1093E20028E4C39BFBE49AFAE499F9E498F8800331
:1093F20012432830D50DE4C39FFFE49EFEE49DFD99
:04940200E49CFC22C8
:1043BA00EB9FF5F0EA9E42F0E99D42F0EC6480C87A
:0643CA0064809845F0221A
:1043D000EB9FF5F0EA9E42F0E99D42F0E89C45F043
:0143E00022BA
:1043E100E8600FECC313FCED13FDEE13FEEF13FFBA
:0343F100D8F122DE
:1043F400E8600FEFC333FFEE33FEED33FDEC33FC27
:03440400D8F122CA
:104407007401FF3395E0FEFDFCA3A3A3E0CF2FF0DB
:10441700E582158270021583E0CE3EF0E5821582B3
:1044270070021583E0CD3DF0E58215827002158399
:05443700E0CC3CF02286
:0C443C00ECF0A3EDF0A3EEF0A3EFF022F3
:10444800A8828583F0D083D08212445F12445F1221
:10445800445F12445FE473E493A3C583C5F0C58346
:10446800C8C582C8F0A3C583C5F0C583C8C582C8BE
:014478002221
:0C447900A42582F582E5F03583F583224E
:10448500D083D082F8E4937012740193700DA3A3C6
:1044950093F8740193F5828883E4737402936860DA
:0644A500EFA3A3A380DFDA
:1044AB00EC8EF0A4CCC5F0CCCDF8EFA4CEC5F02D9E
:1044BB00FDE43CFCE8A42EC8C5F03DFDE43CFCEF5C
:0D44CB00A4FFE5F028FEE43DFDE43CFC22EA
:1044D800EF4E6012EF60010EEDBB010B89828A83FB
:1044E800F0A3DFFCDEFA2289F05007F709DFFCA908
:0C44F800F022BBFEFCF309DFFCA9F0225F
:00000001FF
